 jaccesswalker

 Timestamp is 5a937a1d (reproducible build file hash)

 Preferred load address is 00400000

 Start         Length     Name                   Class
 0001:00000000 00006d90H .text$mn                CODE
 0001:00006d90 00000044H .text$x                 CODE
 0002:00000000 000001c4H .idata$5                DATA
 0002:000001c4 00000008H .00cfg                  DATA
 0002:000001cc 00000004H .CRT$XCA                DATA
 0002:000001d0 00000004H .CRT$XCAA               DATA
 0002:000001d4 00000004H .CRT$XCZ                DATA
 0002:000001d8 00000004H .CRT$XIA                DATA
 0002:000001dc 00000004H .CRT$XIAA               DATA
 0002:000001e0 00000004H .CRT$XIAC               DATA
 0002:000001e4 00000004H .CRT$XIZ                DATA
 0002:000001e8 00000004H .CRT$XPA                DATA
 0002:000001ec 00000004H .CRT$XPZ                DATA
 0002:000001f0 00000004H .CRT$XTA                DATA
 0002:000001f4 00000004H .CRT$XTZ                DATA
 0002:000001f8 00000000H .gfids$y                DATA
 0002:000001f8 00001a08H .rdata                  DATA
 0002:00001c00 00000000H .rdata$CastGuardVftablesA DATA
 0002:00001c00 00000000H .rdata$CastGuardVftablesC DATA
 0002:00001c00 0000012cH .rdata$r                DATA
 0002:00001d2c 00000008H .rdata$sxdata           DATA
 0002:00001d34 000000c4H .rdata$voltmd           DATA
 0002:00001df8 00000318H .rdata$zzzdbg           DATA
 0002:00002110 00000004H .rtc$IAA                DATA
 0002:00002114 00000004H .rtc$IZZ                DATA
 0002:00002118 00000004H .rtc$TAA                DATA
 0002:0000211c 00000004H .rtc$TZZ                DATA
 0002:00002120 000000fcH .xdata$x                DATA
 0002:0000221c 00000000H .edata                  DATA
 0002:0000221c 00000104H .idata$2                DATA
 0002:00002320 00000014H .idata$3                DATA
 0002:00002334 000001c4H .idata$4                DATA
 0002:000024f8 0000083eH .idata$6                DATA
 0003:00000000 00000ad8H .data                   DATA
 0003:00000ad8 00000060H .data$r                 DATA
 0003:00000b38 00000028H .data$rs                DATA
 0003:00000b60 00000690H .bss                    DATA
 0004:00000000 000001d0H .rsrc$01                DATA
 0004:000001d0 00000550H .rsrc$02                DATA

  Address         Publics by Value              Rva+Base       Lib:Object

 0000:00000000       ___AbsoluteZero            00000000     <absolute>
 0000:00000000       ___arm64x_extra_rfe_table  00000000     <absolute>
 0000:00000000       ___arm64x_extra_rfe_table_size 00000000     <absolute>
 0000:00000000       ___arm64x_native_entrypoint 00000000     <absolute>
 0000:00000000       ___arm64x_redirection_metadata 00000000     <absolute>
 0000:00000000       ___arm64x_redirection_metadata_count 00000000     <absolute>
 0000:00000000       ___dynamic_value_reloc_table 00000000     <absolute>
 0000:00000000       ___enclave_config          00000000     <absolute>
 0000:00000000       ___guard_check_icall_a64n_fptr 00000000     <absolute>
 0000:00000000       ___guard_eh_cont_count     00000000     <absolute>
 0000:00000000       ___guard_eh_cont_table     00000000     <absolute>
 0000:00000000       ___guard_fids_count        00000000     <absolute>
 0000:00000000       ___guard_fids_table        00000000     <absolute>
 0000:00000000       ___guard_iat_count         00000000     <absolute>
 0000:00000000       ___guard_iat_table         00000000     <absolute>
 0000:00000000       ___guard_longjmp_count     00000000     <absolute>
 0000:00000000       ___guard_longjmp_table     00000000     <absolute>
 0000:00000000       ___hybrid_auxiliary_delayload_iat 00000000     <absolute>
 0000:00000000       ___hybrid_auxiliary_delayload_iat_copy 00000000     <absolute>
 0000:00000000       ___hybrid_auxiliary_iat    00000000     <absolute>
 0000:00000000       ___hybrid_auxiliary_iat_copy 00000000     <absolute>
 0000:00000000       ___hybrid_code_map         00000000     <absolute>
 0000:00000000       ___hybrid_code_map_count   00000000     <absolute>
 0000:00000000       ___hybrid_image_info_bitfield 00000000     <absolute>
 0000:00000000       ___x64_code_ranges_to_entry_points 00000000     <absolute>
 0000:00000000       ___x64_code_ranges_to_entry_points_count 00000000     <absolute>
 0000:00000002       ___safe_se_handler_count   00000002     <absolute>
 0000:00000100       ___guard_flags             00000100     <absolute>
 0000:00000000       ___ImageBase               00400000     <linker-defined>
 0001:00000000       _initializeAccessBridge    00401000 f   AccessBridgeCalls.obj
 0001:00000ec0       _shutdownAccessBridge      00401ec0 f   AccessBridgeCalls.obj
 0001:00000f10       _IsJavaWindow              00401f10 f   AccessBridgeCalls.obj
 0001:00000f40       _GetAccessibleContextFromHWND 00401f40 f   AccessBridgeCalls.obj
 0001:00000f70       _getHWNDFromAccessibleContext 00401f70 f   AccessBridgeCalls.obj
 0001:00000fa0       _SetJavaShutdown           00401fa0 f   AccessBridgeCalls.obj
 0001:00000fc0       _SetFocusGained            00401fc0 f   AccessBridgeCalls.obj
 0001:00000fe0       _SetFocusLost              00401fe0 f   AccessBridgeCalls.obj
 0001:00001000       _SetCaretUpdate            00402000 f   AccessBridgeCalls.obj
 0001:00001020       _SetMouseClicked           00402020 f   AccessBridgeCalls.obj
 0001:00001040       _SetMouseEntered           00402040 f   AccessBridgeCalls.obj
 0001:00001060       _SetMouseExited            00402060 f   AccessBridgeCalls.obj
 0001:00001080       _SetMousePressed           00402080 f   AccessBridgeCalls.obj
 0001:000010a0       _SetMouseReleased          004020a0 f   AccessBridgeCalls.obj
 0001:000010c0       _SetMenuCanceled           004020c0 f   AccessBridgeCalls.obj
 0001:000010e0       _SetMenuDeselected         004020e0 f   AccessBridgeCalls.obj
 0001:00001100       _SetMenuSelected           00402100 f   AccessBridgeCalls.obj
 0001:00001120       _SetPopupMenuCanceled      00402120 f   AccessBridgeCalls.obj
 0001:00001140       _SetPopupMenuWillBecomeInvisible 00402140 f   AccessBridgeCalls.obj
 0001:00001160       _SetPopupMenuWillBecomeVisible 00402160 f   AccessBridgeCalls.obj
 0001:00001180       _SetPropertyNameChange     00402180 f   AccessBridgeCalls.obj
 0001:000011a0       _SetPropertyDescriptionChange 004021a0 f   AccessBridgeCalls.obj
 0001:000011c0       _SetPropertyStateChange    004021c0 f   AccessBridgeCalls.obj
 0001:000011e0       _SetPropertyValueChange    004021e0 f   AccessBridgeCalls.obj
 0001:00001200       _SetPropertySelectionChange 00402200 f   AccessBridgeCalls.obj
 0001:00001220       _SetPropertyTextChange     00402220 f   AccessBridgeCalls.obj
 0001:00001240       _SetPropertyCaretChange    00402240 f   AccessBridgeCalls.obj
 0001:00001260       _SetPropertyVisibleDataChange 00402260 f   AccessBridgeCalls.obj
 0001:00001280       _SetPropertyChildChange    00402280 f   AccessBridgeCalls.obj
 0001:000012a0       _SetPropertyActiveDescendentChange 004022a0 f   AccessBridgeCalls.obj
 0001:000012c0       _SetPropertyTableModelChange 004022c0 f   AccessBridgeCalls.obj
 0001:000012e0       _ReleaseJavaObject         004022e0 f   AccessBridgeCalls.obj
 0001:00001300       _GetVersionInfo            00402300 f   AccessBridgeCalls.obj
 0001:00001330       _GetAccessibleContextAt    00402330 f   AccessBridgeCalls.obj
 0001:00001360       _GetAccessibleContextWithFocus 00402360 f   AccessBridgeCalls.obj
 0001:00001390       _GetAccessibleContextInfo  00402390 f   AccessBridgeCalls.obj
 0001:000013c0       _GetAccessibleChildFromContext 004023c0 f   AccessBridgeCalls.obj
 0001:000013f0       _GetAccessibleParentFromContext 004023f0 f   AccessBridgeCalls.obj
 0001:00001420       _GetAccessibleTextInfo     00402420 f   AccessBridgeCalls.obj
 0001:00001450       _GetAccessibleTextItems    00402450 f   AccessBridgeCalls.obj
 0001:00001480       _GetAccessibleTextSelectionInfo 00402480 f   AccessBridgeCalls.obj
 0001:000014b0       _GetAccessibleTextAttributes 004024b0 f   AccessBridgeCalls.obj
 0001:000014e0       _GetAccessibleTextRect     004024e0 f   AccessBridgeCalls.obj
 0001:00001510       _GetAccessibleTextLineBounds 00402510 f   AccessBridgeCalls.obj
 0001:00001540       _GetAccessibleTextRange    00402540 f   AccessBridgeCalls.obj
 0001:00001580       _getAccessibleTableInfo    00402580 f   AccessBridgeCalls.obj
 0001:000015b0       _getAccessibleTableCellInfo 004025b0 f   AccessBridgeCalls.obj
 0001:000015e0       _getAccessibleTableRowHeader 004025e0 f   AccessBridgeCalls.obj
 0001:00001610       _getAccessibleTableColumnHeader 00402610 f   AccessBridgeCalls.obj
 0001:00001640       _getAccessibleTableRowDescription 00402640 f   AccessBridgeCalls.obj
 0001:00001670       _getAccessibleTableColumnDescription 00402670 f   AccessBridgeCalls.obj
 0001:000016a0       _getAccessibleTableRowSelectionCount 004026a0 f   AccessBridgeCalls.obj
 0001:000016d0       _isAccessibleTableRowSelected 004026d0 f   AccessBridgeCalls.obj
 0001:00001700       _getAccessibleTableRowSelections 00402700 f   AccessBridgeCalls.obj
 0001:00001730       _getAccessibleTableColumnSelectionCount 00402730 f   AccessBridgeCalls.obj
 0001:00001760       _isAccessibleTableColumnSelected 00402760 f   AccessBridgeCalls.obj
 0001:00001790       _getAccessibleTableColumnSelections 00402790 f   AccessBridgeCalls.obj
 0001:000017c0       _getAccessibleTableRow     004027c0 f   AccessBridgeCalls.obj
 0001:000017f0       _getAccessibleTableColumn  004027f0 f   AccessBridgeCalls.obj
 0001:00001820       _getAccessibleTableIndex   00402820 f   AccessBridgeCalls.obj
 0001:00001850       _getAccessibleRelationSet  00402850 f   AccessBridgeCalls.obj
 0001:00001880       _getAccessibleHypertext    00402880 f   AccessBridgeCalls.obj
 0001:000018b0       _activateAccessibleHyperlink 004028b0 f   AccessBridgeCalls.obj
 0001:000018e0       _getAccessibleHyperlinkCount 004028e0 f   AccessBridgeCalls.obj
 0001:00001910       _getAccessibleHypertextExt 00402910 f   AccessBridgeCalls.obj
 0001:00001940       _getAccessibleHypertextLinkIndex 00402940 f   AccessBridgeCalls.obj
 0001:00001970       _getAccessibleHyperlink    00402970 f   AccessBridgeCalls.obj
 0001:000019a0       _getAccessibleKeyBindings  004029a0 f   AccessBridgeCalls.obj
 0001:000019d0       _getAccessibleIcons        004029d0 f   AccessBridgeCalls.obj
 0001:00001a00       _getAccessibleActions      00402a00 f   AccessBridgeCalls.obj
 0001:00001a30       _doAccessibleActions       00402a30 f   AccessBridgeCalls.obj
 0001:00001a60       _IsSameObject              00402a60 f   AccessBridgeCalls.obj
 0001:00001a90       _setTextContents           00402a90 f   AccessBridgeCalls.obj
 0001:00001ac0       _getParentWithRole         00402ac0 f   AccessBridgeCalls.obj
 0001:00001af0       _getParentWithRoleElseRoot 00402af0 f   AccessBridgeCalls.obj
 0001:00001b20       _getTopLevelObject         00402b20 f   AccessBridgeCalls.obj
 0001:00001b50       _getObjectDepth            00402b50 f   AccessBridgeCalls.obj
 0001:00001b80       _getActiveDescendent       00402b80 f   AccessBridgeCalls.obj
 0001:00001bb0       _GetCurrentAccessibleValueFromContext 00402bb0 f   AccessBridgeCalls.obj
 0001:00001be0       _GetMaximumAccessibleValueFromContext 00402be0 f   AccessBridgeCalls.obj
 0001:00001c10       _GetMinimumAccessibleValueFromContext 00402c10 f   AccessBridgeCalls.obj
 0001:00001c40       _GetAccessibleSelectionFromContext 00402c40 f   AccessBridgeCalls.obj
 0001:00001c70       _GetAccessibleSelectionCountFromContext 00402c70 f   AccessBridgeCalls.obj
 0001:00001ca0       _IsAccessibleChildSelectedFromContext 00402ca0 f   AccessBridgeCalls.obj
 0001:00001cd0       _RemoveAccessibleSelectionFromContext 00402cd0 f   AccessBridgeCalls.obj
 0001:00001d00       _SelectAllAccessibleSelectionFromContext 00402d00 f   AccessBridgeCalls.obj
 0001:00001d20       _getVirtualAccessibleName  00402d20 f   AccessBridgeCalls.obj
 0001:00001d50       _requestFocus              00402d50 f   AccessBridgeCalls.obj
 0001:00001d80       _selectTextRange           00402d80 f   AccessBridgeCalls.obj
 0001:00001db0       _getTextAttributesInRange  00402db0 f   AccessBridgeCalls.obj
 0001:00001df0       _getVisibleChildrenCount   00402df0 f   AccessBridgeCalls.obj
 0001:00001e20       _getVisibleChildren        00402e20 f   AccessBridgeCalls.obj
 0001:00001e50       _setCaretPosition          00402e50 f   AccessBridgeCalls.obj
 0001:00001e80       _getCaretLocation          00402e80 f   AccessBridgeCalls.obj
 0001:00001eb0       _getEventsWaiting          00402eb0 f   AccessBridgeCalls.obj
 0001:00001ed0       _addAccessibleSelectionFromContext 00402ed0 f   AccessBridgeCalls.obj
 0001:00001f00       _clearAccessibleSelectionFromContext 00402f00 f   AccessBridgeCalls.obj
 0001:00001f20       _printError                00402f20 f   AccessBridgeDebug.obj
 0001:00002030       _PrintDebugString          00403030 f   AccessBridgeDebug.obj
 0001:000020a0       _wPrintJavaDebugString     004030a0 f   AccessBridgeDebug.obj
 0001:00002110       _wPrintDebugString         00403110 f   AccessBridgeDebug.obj
 0001:00002180       _initializeFileLogger      00403180 f   AccessBridgeDebug.obj
 0001:000022b0       _finalizeFileLogger        004032b0 f   AccessBridgeDebug.obj
 0001:000022e0       _getTimeStamp              004032e0 f   AccessBridgeDebug.obj
 0001:00002320       _PrintJavaDebugString2     00403320 f   AccessBridgeDebug.obj
 0001:00002390       ___local_stdio_printf_options 00403390 f i AccessBridgeDebug.obj
 0001:000023a0       __vfprintf_l               004033a0 f i AccessBridgeDebug.obj
 0001:000023d0       __vfwprintf_l              004033d0 f i AccessBridgeDebug.obj
 0001:00002400       _fprintf                   00403400 f i AccessBridgeDebug.obj
 0001:00002440       _printf                    00403440 f i AccessBridgeDebug.obj
 0001:00002480       _vfprintf                  00403480 f i AccessBridgeDebug.obj
 0001:000024a0       _vfwprintf                 004034a0 f i AccessBridgeDebug.obj
 0001:000024c0       ?initBroadcastMessageIDs@@YAHXZ 004034c0 f   AccessBridgeMessages.obj
 0001:00002510       ?getTimeAndDate@@YAPADXZ   00403510 f   AccessInfo.obj
 0001:000025c0       ?displayAndLog@@YAXPAUHWND__@@HPAU_iobuf@@PADZZ 004035c0 f   AccessInfo.obj
 0001:000026a0       ?logString@@YAXPAU_iobuf@@PADZZ 004036a0 f   AccessInfo.obj
 0001:00002730       ?getAccessibleInfo@@YAPADJPAV_jobject@@PADH@Z 00403730 f   AccessInfo.obj
 0001:00002760       ?getAccessibleInfo@@YAPADJPAV_jobject@@HHPADH@Z 00403760 f   AccessInfo.obj
 0001:000047f0       ?appendToBuffer@@YAHPADI0ZZ 004057f0 f   AccessInfo.obj
 0001:000048d0       _snprintf                  004058d0 f i AccessInfo.obj
 0001:00004910       _vsnprintf                 00405910 f i AccessInfo.obj
 0001:00004960       _WinMain@16                00405960 f   jaccesswalker.obj
 0001:000049f0       ??0AccessibleNode@@QAE@JPAV_jobject@@PAV0@PAUHWND__@@PAU_TREEITEM@@@Z 004059f0 f   jaccesswalker.obj
 0001:00004a30       ??1AccessibleNode@@QAE@XZ  00405a30 f   jaccesswalker.obj
 0001:00004a60       ?setAccessibleName@AccessibleNode@@QAEXPAD@Z 00405a60 f   jaccesswalker.obj
 0001:00004a90       ?setAccessibleRole@AccessibleNode@@QAEXPAD@Z 00405a90 f   jaccesswalker.obj
 0001:00004ac0       ?displayAPIWindow@AccessibleNode@@QAEHXZ 00405ac0 f   jaccesswalker.obj
 0001:00004be0       ??0Jaccesswalker@@QAE@H@Z  00405be0 f   jaccesswalker.obj
 0001:00004da0       ?buildAccessibilityTree@Jaccesswalker@@QAEXXZ 00405da0 f   jaccesswalker.obj
 0001:00004dd0       ?addComponentNodes@Jaccesswalker@@QAEXJPAV_jobject@@PAVAccessibleNode@@PAUHWND__@@PAU_TREEITEM@@2@Z 00405dd0 f   jaccesswalker.obj
 0001:000050c0       ?WinProc@@YGJPAUHWND__@@IIJ@Z 004060c0 f   jaccesswalker.obj
 0001:00005390       ?EnumWndProc@@YGHPAUHWND__@@J@Z 00406390 f   jaccesswalker.obj
 0001:00005490       ?EnumChildProc@@YGHPAUHWND__@@J@Z 00406490 f   jaccesswalker.obj
 0001:00005530       ?CreateATreeView@@YAPAUHWND__@@PAU1@@Z 00406530 f   jaccesswalker.obj
 0001:000055a0       ?AccessInfoWindowProc@@YGJPAUHWND__@@IIJ@Z 004065a0 f   jaccesswalker.obj
 0001:000056a0       ?IsInaccessibleJavaWindow@@YAHQAUHWND__@@@Z 004066a0 f   jaccesswalker.obj
 0001:00005da2       ??_U@YAPAXI@Z              00406da2 f   MSVCRT:new_array.obj
 0001:00005dab       ??_V@YAXPAX@Z              00406dab f   MSVCRT:delete_array.obj
 0001:00005db0       ___raise_securityfailure   00406db0 f   MSVCRT:gs_report.obj
 0001:00005dd8       ___report_gsfailure        00406dd8 f   MSVCRT:gs_report.obj
 0001:00005ed2       ___report_rangecheckfailure 00406ed2 f   MSVCRT:gs_report.obj
 0001:00005ede       ___report_securityfailure  00406ede f   MSVCRT:gs_report.obj
 0001:00005fb0       __aulldiv                  00406fb0 f   MSVCRT:ulldiv.obj
 0001:00006018       @__security_check_cookie@4 00407018 f   MSVCRT:secchk.obj
 0001:00006030       __alloca_probe             00407030 f   MSVCRT:chkstk.obj
 0001:00006030       __chkstk                   00407030 f   MSVCRT:chkstk.obj
 0001:0000605b       ??2@YAPAXI@Z               0040705b f   MSVCRT:new_scalar.obj
 0001:0000608b       ??3@YAXPAXI@Z              0040708b f   MSVCRT:delete_scalar_size.obj
 0001:000062da       _WinMainCRTStartup         004072da f   MSVCRT:exe_winmain.obj
 0001:000062e4       ??3@YAXPAX@Z               004072e4 f   MSVCRT:delete_scalar.obj
 0001:000062e9       ??0bad_alloc@std@@QAE@ABV01@@Z 004072e9 f i MSVCRT:throw_bad_alloc.obj
 0001:00006304       ??0bad_alloc@std@@QAE@XZ   00407304 f i MSVCRT:throw_bad_alloc.obj
 0001:0000631c       ??0bad_array_new_length@std@@QAE@ABV01@@Z 0040731c f i MSVCRT:throw_bad_alloc.obj
 0001:00006337       ??0bad_array_new_length@std@@QAE@XZ 00407337 f i MSVCRT:throw_bad_alloc.obj
 0001:0000634f       ??0exception@std@@QAE@ABV01@@Z 0040734f f i MSVCRT:throw_bad_alloc.obj
 0001:0000637b       ??1bad_alloc@std@@UAE@XZ   0040737b f i MSVCRT:throw_bad_alloc.obj
 0001:0000637b       ??1bad_array_new_length@std@@UAE@XZ 0040737b f i MSVCRT:throw_bad_alloc.obj
 0001:0000638c       ??_Ebad_alloc@std@@UAEPAXI@Z 0040738c f i MSVCRT:throw_bad_alloc.obj
 0001:0000638c       ??_Ebad_array_new_length@std@@UAEPAXI@Z 0040738c f i MSVCRT:throw_bad_alloc.obj
 0001:0000638c       ??_Eexception@std@@UAEPAXI@Z 0040738c f i MSVCRT:throw_bad_alloc.obj
 0001:0000638c       ??_Gbad_alloc@std@@UAEPAXI@Z 0040738c f i MSVCRT:throw_bad_alloc.obj
 0001:0000638c       ??_Gbad_array_new_length@std@@UAEPAXI@Z 0040738c f i MSVCRT:throw_bad_alloc.obj
 0001:0000638c       ??_Gexception@std@@UAEPAXI@Z 0040738c f i MSVCRT:throw_bad_alloc.obj
 0001:000063b9       ?__scrt_throw_std_bad_alloc@@YAXXZ 004073b9 f   MSVCRT:throw_bad_alloc.obj
 0001:000063d6       ?__scrt_throw_std_bad_array_new_length@@YAXXZ 004073d6 f   MSVCRT:throw_bad_alloc.obj
 0001:000063f3       ?what@exception@std@@UBEPBDXZ 004073f3 f i MSVCRT:throw_bad_alloc.obj
 0001:00006444       ___scrt_acquire_startup_lock 00407444 f   MSVCRT:utility.obj
 0001:00006476       ___scrt_initialize_crt     00407476 f   MSVCRT:utility.obj
 0001:000064af       ___scrt_initialize_onexit_tables 004074af f   MSVCRT:utility.obj
 0001:00006536       ___scrt_is_nonwritable_in_current_image 00407536 f   MSVCRT:utility.obj
 0001:000065ca       ___scrt_release_startup_lock 004075ca f   MSVCRT:utility.obj
 0001:000065e7       ___scrt_uninitialize_crt   004075e7 f   MSVCRT:utility.obj
 0001:0000660f       __onexit                   0040760f f   MSVCRT:utility.obj
 0001:0000663c       _atexit                    0040763c f   MSVCRT:utility.obj
 0001:0000669e       ___security_init_cookie    0040769e f   MSVCRT:gs_support.obj
 0001:000066e9       ___scrt_exe_initialize_mta 004076e9 f   MSVCRT:utility_desktop.obj
 0001:000066e9       ___scrt_initialize_winrt   004076e9 f   MSVCRT:utility_desktop.obj
 0001:000066e9       ___scrt_stub_for_initialize_mta 004076e9 f   MSVCRT:utility_desktop.obj
 0001:000066e9       __get_startup_commit_mode  004076e9 f   MSVCRT:commit_mode.obj
 0001:000066e9       __get_startup_new_mode     004076e9 f   MSVCRT:new_mode.obj
 0001:000066e9       __get_startup_thread_locale_mode 004076e9 f   MSVCRT:thread_locale.obj
 0001:000066e9       __matherr                  004076e9 f   MSVCRT:matherr.obj
 0001:000066ec       __get_startup_argv_mode    004076ec f   MSVCRT:argv_mode.obj
 0001:000066f0       __get_startup_file_mode    004076f0 f   MSVCRT:file_mode.obj
 0001:000066f6       ?__scrt_initialize_type_info@@YAXXZ 004076f6 f   MSVCRT:tncleanup.obj
 0001:00006702       ___acrt_initialize         00407702 f   MSVCRT:ucrt_stubs.obj
 0001:00006702       ___acrt_uninitialize       00407702 f   MSVCRT:ucrt_stubs.obj
 0001:00006702       ___scrt_stub_for_acrt_initialize 00407702 f   MSVCRT:ucrt_stubs.obj
 0001:00006702       ___scrt_stub_for_acrt_uninitialize 00407702 f   MSVCRT:ucrt_stubs.obj
 0001:00006702       ___vcrt_initialize         00407702 f   MSVCRT:ucrt_stubs.obj
 0001:00006702       ___vcrt_uninitialize       00407702 f   MSVCRT:ucrt_stubs.obj
 0001:00006702       __should_initialize_environment 00407702 f   MSVCRT:env_mode.obj
 0001:00006705       __initialize_default_precision 00407705 f   MSVCRT:default_precision.obj
 0001:00006726       @_guard_check_icall_nop@4  00407726 f   MSVCRT:guard_support.obj
 0001:00006726       __initialize_denormal_control 00407726 f   MSVCRT:denormal_control.obj
 0001:00006726       __initialize_invalid_parameter_handler 00407726 f   MSVCRT:invalid_parameter_handler.obj
 0001:00006729       ___local_stdio_scanf_options 00407729 f i MSVCRT:default_local_stdio_options.obj
 0001:0000672f       ___scrt_initialize_default_local_stdio_options 0040772f f   MSVCRT:default_local_stdio_options.obj
 0001:0000674c       ___scrt_is_user_matherr_present 0040774c f   MSVCRT:matherr_detection.obj
 0001:00006758       ___scrt_get_dyn_tls_init_callback 00407758 f   MSVCRT:dyn_tls_init.obj
 0001:0000675e       ___scrt_get_dyn_tls_dtor_callback 0040775e f   MSVCRT:dyn_tls_dtor.obj
 0001:00006764       ___scrt_fastfail           00407764 f   MSVCRT:utility_desktop.obj
 0001:0000687f       ___scrt_get_show_window_mode 0040787f f   MSVCRT:utility_desktop.obj
 0001:000068b0       ___scrt_initialize_mta     004078b0 f   MSVCRT:utility_desktop.obj
 0001:000068b5       ___scrt_is_managed_app     004078b5 f   MSVCRT:utility_desktop.obj
 0001:000068f7       ___scrt_set_unhandled_exception_filter 004078f7 f   MSVCRT:utility_desktop.obj
 0001:00006903       ___scrt_unhandled_exception_filter@4 00407903 f   MSVCRT:utility_desktop.obj
 0001:00006959       __crt_debugger_hook        00407959 f   MSVCRT:utility_desktop.obj
 0001:00006961       __RTC_Initialize           00407961 f   MSVCRT:initsect.obj
 0001:0000698d       __RTC_Terminate            0040798d f   MSVCRT:initsect.obj
 0001:000069c0       __SEH_prolog4              004079c0 f   MSVCRT:sehprolg4.obj
 0001:00006a05       __except_handler4          00407a05 f   MSVCRT:chandler4gs.obj
 0001:00006a34       ??_Etype_info@@UAEPAXI@Z   00407a34 f i MSVCRT:std_type_info_static.obj
 0001:00006a34       ??_Gtype_info@@UAEPAXI@Z   00407a34 f i MSVCRT:std_type_info_static.obj
 0001:00006a57       ___isa_available_init      00407a57 f   MSVCRT:cpu_disp.obj
 0001:00006c2b       ___scrt_is_ucrt_dll_in_use 00407c2b f   MSVCRT:ucrt_detection.obj
 0001:00006c37       _memcpy                    00407c37 f   vcruntime:VCRUNTIME140.dll
 0001:00006c3d       _memset                    00407c3d f   vcruntime:VCRUNTIME140.dll
 0001:00006c43       ___CxxFrameHandler3        00407c43 f   vcruntime:VCRUNTIME140.dll
 0001:00006c49       ___std_exception_copy      00407c49 f   vcruntime:VCRUNTIME140.dll
 0001:00006c4f       ___std_exception_destroy   00407c4f f   vcruntime:VCRUNTIME140.dll
 0001:00006c55       __CxxThrowException@8      00407c55 f   vcruntime:VCRUNTIME140.dll
 0001:00006c5b       ___current_exception       00407c5b f   vcruntime:VCRUNTIME140.dll
 0001:00006c61       ___current_exception_context 00407c61 f   vcruntime:VCRUNTIME140.dll
 0001:00006c67       __except_handler4_common   00407c67 f   vcruntime:VCRUNTIME140.dll
 0001:00006c6d       _strlen                    00407c6d f   ucrt:api-ms-win-crt-string-l1-1-0.dll
 0001:00006c73       _strcpy                    00407c73 f   ucrt:api-ms-win-crt-string-l1-1-0.dll
 0001:00006c79       _strcmp                    00407c79 f   ucrt:api-ms-win-crt-string-l1-1-0.dll
 0001:00006c7f       __callnewh                 00407c7f f   ucrt:api-ms-win-crt-heap-l1-1-0.dll
 0001:00006c85       _malloc                    00407c85 f   ucrt:api-ms-win-crt-heap-l1-1-0.dll
 0001:00006c8b       __seh_filter_exe           00407c8b f   ucrt:api-ms-win-crt-runtime-l1-1-0.dll
 0001:00006c91       __set_app_type             00407c91 f   ucrt:api-ms-win-crt-runtime-l1-1-0.dll
 0001:00006c97       ___setusermatherr          00407c97 f   ucrt:api-ms-win-crt-math-l1-1-0.dll
 0001:00006c9d       __configure_narrow_argv    00407c9d f   ucrt:api-ms-win-crt-runtime-l1-1-0.dll
 0001:00006ca3       __initialize_narrow_environment 00407ca3 f   ucrt:api-ms-win-crt-runtime-l1-1-0.dll
 0001:00006ca9       __get_narrow_winmain_command_line 00407ca9 f   ucrt:api-ms-win-crt-runtime-l1-1-0.dll
 0001:00006caf       __initterm                 00407caf f   ucrt:api-ms-win-crt-runtime-l1-1-0.dll
 0001:00006cb5       __initterm_e               00407cb5 f   ucrt:api-ms-win-crt-runtime-l1-1-0.dll
 0001:00006cbb       _exit                      00407cbb f   ucrt:api-ms-win-crt-runtime-l1-1-0.dll
 0001:00006cc1       __exit                     00407cc1 f   ucrt:api-ms-win-crt-runtime-l1-1-0.dll
 0001:00006cc7       __set_fmode                00407cc7 f   ucrt:api-ms-win-crt-stdio-l1-1-0.dll
 0001:00006ccd       __cexit                    00407ccd f   ucrt:api-ms-win-crt-runtime-l1-1-0.dll
 0001:00006cd3       __c_exit                   00407cd3 f   ucrt:api-ms-win-crt-runtime-l1-1-0.dll
 0001:00006cd9       __register_thread_local_exe_atexit_callback 00407cd9 f   ucrt:api-ms-win-crt-runtime-l1-1-0.dll
 0001:00006cdf       __configthreadlocale       00407cdf f   ucrt:api-ms-win-crt-locale-l1-1-0.dll
 0001:00006ce5       __set_new_mode             00407ce5 f   ucrt:api-ms-win-crt-heap-l1-1-0.dll
 0001:00006ceb       ___p__commode              00407ceb f   ucrt:api-ms-win-crt-stdio-l1-1-0.dll
 0001:00006cf1       _free                      00407cf1 f   ucrt:api-ms-win-crt-heap-l1-1-0.dll
 0001:00006cf7       __initialize_onexit_table  00407cf7 f   ucrt:api-ms-win-crt-runtime-l1-1-0.dll
 0001:00006cfd       __register_onexit_function 00407cfd f   ucrt:api-ms-win-crt-runtime-l1-1-0.dll
 0001:00006d03       __crt_atexit               00407d03 f   ucrt:api-ms-win-crt-runtime-l1-1-0.dll
 0001:00006d09       __controlfp_s              00407d09 f   ucrt:api-ms-win-crt-runtime-l1-1-0.dll
 0001:00006d0f       _terminate                 00407d0f f   ucrt:api-ms-win-crt-runtime-l1-1-0.dll
 0001:00006d15       __filter_x86_sse2_floating_point_exception 00407d15 f   MSVCRT:x86_exception_filter.obj
 0001:00006d15       __filter_x86_sse2_floating_point_exception_default 00407d15 f   MSVCRT:x86_exception_filter.obj
 0002:00000000       __imp__InitCommonControlsEx@4 00408000     comctl32:COMCTL32.dll
 0002:00000004       \177COMCTL32_NULL_THUNK_DATA 00408004     comctl32:COMCTL32.dll
 0002:00000008       __imp__GetStockObject@4    00408008     gdi32:GDI32.dll
 0002:0000000c       \177GDI32_NULL_THUNK_DATA  0040800c     gdi32:GDI32.dll
 0002:00000010       __imp__GetModuleHandleW@4  00408010     kernel32:KERNEL32.dll
 0002:00000014       __imp__GetStartupInfoW@4   00408014     kernel32:KERNEL32.dll
 0002:00000018       __imp__IsDebuggerPresent@0 00408018     kernel32:KERNEL32.dll
 0002:0000001c       __imp__InitializeSListHead@4 0040801c     kernel32:KERNEL32.dll
 0002:00000020       __imp__GetCurrentThreadId@0 00408020     kernel32:KERNEL32.dll
 0002:00000024       __imp__GetCurrentProcessId@0 00408024     kernel32:KERNEL32.dll
 0002:00000028       __imp__QueryPerformanceCounter@4 00408028     kernel32:KERNEL32.dll
 0002:0000002c       __imp__IsProcessorFeaturePresent@4 0040802c     kernel32:KERNEL32.dll
 0002:00000030       __imp__TerminateProcess@8  00408030     kernel32:KERNEL32.dll
 0002:00000034       __imp__GetCurrentProcess@0 00408034     kernel32:KERNEL32.dll
 0002:00000038       __imp__SetUnhandledExceptionFilter@4 00408038     kernel32:KERNEL32.dll
 0002:0000003c       __imp__UnhandledExceptionFilter@4 0040803c     kernel32:KERNEL32.dll
 0002:00000040       __imp__FormatMessageA@28   00408040     kernel32:KERNEL32.dll
 0002:00000044       __imp__LocalFree@4         00408044     kernel32:KERNEL32.dll
 0002:00000048       __imp__GetSystemTimeAsFileTime@4 00408048     kernel32:KERNEL32.dll
 0002:0000004c       __imp__LoadLibraryA@4      0040804c     kernel32:KERNEL32.dll
 0002:00000050       __imp__GetProcAddress@8    00408050     kernel32:KERNEL32.dll
 0002:00000054       __imp__FreeLibrary@4       00408054     kernel32:KERNEL32.dll
 0002:00000058       __imp__GetLastError@0      00408058     kernel32:KERNEL32.dll
 0002:0000005c       \177KERNEL32_NULL_THUNK_DATA 0040805c     kernel32:KERNEL32.dll
 0002:00000060       __imp__GetClientRect@8     00408060     user32:USER32.dll
 0002:00000064       __imp__GetCursorPos@4      00408064     user32:USER32.dll
 0002:00000068       __imp__UpdateWindow@4      00408068     user32:USER32.dll
 0002:0000006c       __imp__EnumChildWindows@12 0040806c     user32:USER32.dll
 0002:00000070       __imp__EnumWindows@8       00408070     user32:USER32.dll
 0002:00000074       __imp__GetClassNameA@12    00408074     user32:USER32.dll
 0002:00000078       __imp__LoadCursorA@8       00408078     user32:USER32.dll
 0002:0000007c       __imp__LoadIconA@8         0040807c     user32:USER32.dll
 0002:00000080       __imp__RegisterWindowMessageA@4 00408080     user32:USER32.dll
 0002:00000084       __imp__TrackPopupMenu@28   00408084     user32:USER32.dll
 0002:00000088       __imp__GetSubMenu@8        00408088     user32:USER32.dll
 0002:0000008c       __imp__LoadMenuA@8         0040808c     user32:USER32.dll
 0002:00000090       __imp__GetDlgItem@8        00408090     user32:USER32.dll
 0002:00000094       __imp__EndDialog@8         00408094     user32:USER32.dll
 0002:00000098       __imp__SetWindowPos@28     00408098     user32:USER32.dll
 0002:0000009c       __imp__ShowWindow@8        0040809c     user32:USER32.dll
 0002:000000a0       __imp__DestroyWindow@4     004080a0     user32:USER32.dll
 0002:000000a4       __imp__CreateWindowExA@48  004080a4     user32:USER32.dll
 0002:000000a8       __imp__RegisterClassExA@4  004080a8     user32:USER32.dll
 0002:000000ac       __imp__PostQuitMessage@4   004080ac     user32:USER32.dll
 0002:000000b0       __imp__DefWindowProcA@16   004080b0     user32:USER32.dll
 0002:000000b4       __imp__SendMessageA@16     004080b4     user32:USER32.dll
 0002:000000b8       __imp__DispatchMessageA@4  004080b8     user32:USER32.dll
 0002:000000bc       __imp__TranslateMessage@4  004080bc     user32:USER32.dll
 0002:000000c0       __imp__GetMessageA@16      004080c0     user32:USER32.dll
 0002:000000c4       __imp__wsprintfA           004080c4     user32:USER32.dll
 0002:000000c8       __imp__SetDlgItemTextA@12  004080c8     user32:USER32.dll
 0002:000000cc       __imp__ScreenToClient@8    004080cc     user32:USER32.dll
 0002:000000d0       \177USER32_NULL_THUNK_DATA 004080d0     user32:USER32.dll
 0002:000000d4       __imp__memcpy              004080d4     vcruntime:VCRUNTIME140.dll
 0002:000000d8       __imp__memset              004080d8     vcruntime:VCRUNTIME140.dll
 0002:000000dc       __imp____CxxFrameHandler3  004080dc     vcruntime:VCRUNTIME140.dll
 0002:000000e0       __imp____std_exception_copy 004080e0     vcruntime:VCRUNTIME140.dll
 0002:000000e4       __imp____std_exception_destroy 004080e4     vcruntime:VCRUNTIME140.dll
 0002:000000e8       __imp___CxxThrowException@8 004080e8     vcruntime:VCRUNTIME140.dll
 0002:000000ec       __imp____current_exception 004080ec     vcruntime:VCRUNTIME140.dll
 0002:000000f0       __imp____current_exception_context 004080f0     vcruntime:VCRUNTIME140.dll
 0002:000000f4       __imp___except_handler4_common 004080f4     vcruntime:VCRUNTIME140.dll
 0002:000000f8       \177VCRUNTIME140_NULL_THUNK_DATA 004080f8     vcruntime:VCRUNTIME140.dll
 0002:000000fc       __imp__getenv              004080fc     ucrt:api-ms-win-crt-environment-l1-1-0.dll
 0002:00000100       \177api-ms-win-crt-environment-l1-1-0_NULL_THUNK_DATA 00408100     ucrt:api-ms-win-crt-environment-l1-1-0.dll
 0002:00000104       __imp___set_new_mode       00408104     ucrt:api-ms-win-crt-heap-l1-1-0.dll
 0002:00000108       __imp__malloc              00408108     ucrt:api-ms-win-crt-heap-l1-1-0.dll
 0002:0000010c       __imp___callnewh           0040810c     ucrt:api-ms-win-crt-heap-l1-1-0.dll
 0002:00000110       __imp__free                00408110     ucrt:api-ms-win-crt-heap-l1-1-0.dll
 0002:00000114       \177api-ms-win-crt-heap-l1-1-0_NULL_THUNK_DATA 00408114     ucrt:api-ms-win-crt-heap-l1-1-0.dll
 0002:00000118       __imp___configthreadlocale 00408118     ucrt:api-ms-win-crt-locale-l1-1-0.dll
 0002:0000011c       \177api-ms-win-crt-locale-l1-1-0_NULL_THUNK_DATA 0040811c     ucrt:api-ms-win-crt-locale-l1-1-0.dll
 0002:00000120       __imp____setusermatherr    00408120     ucrt:api-ms-win-crt-math-l1-1-0.dll
 0002:00000124       \177api-ms-win-crt-math-l1-1-0_NULL_THUNK_DATA 00408124     ucrt:api-ms-win-crt-math-l1-1-0.dll
 0002:00000128       __imp__terminate           00408128     ucrt:api-ms-win-crt-runtime-l1-1-0.dll
 0002:0000012c       __imp___controlfp_s        0040812c     ucrt:api-ms-win-crt-runtime-l1-1-0.dll
 0002:00000130       __imp___crt_atexit         00408130     ucrt:api-ms-win-crt-runtime-l1-1-0.dll
 0002:00000134       __imp___register_onexit_function 00408134     ucrt:api-ms-win-crt-runtime-l1-1-0.dll
 0002:00000138       __imp___initialize_onexit_table 00408138     ucrt:api-ms-win-crt-runtime-l1-1-0.dll
 0002:0000013c       __imp___seh_filter_exe     0040813c     ucrt:api-ms-win-crt-runtime-l1-1-0.dll
 0002:00000140       __imp___set_app_type       00408140     ucrt:api-ms-win-crt-runtime-l1-1-0.dll
 0002:00000144       __imp___c_exit             00408144     ucrt:api-ms-win-crt-runtime-l1-1-0.dll
 0002:00000148       __imp___configure_narrow_argv 00408148     ucrt:api-ms-win-crt-runtime-l1-1-0.dll
 0002:0000014c       __imp___initialize_narrow_environment 0040814c     ucrt:api-ms-win-crt-runtime-l1-1-0.dll
 0002:00000150       __imp___get_narrow_winmain_command_line 00408150     ucrt:api-ms-win-crt-runtime-l1-1-0.dll
 0002:00000154       __imp___initterm           00408154     ucrt:api-ms-win-crt-runtime-l1-1-0.dll
 0002:00000158       __imp___register_thread_local_exe_atexit_callback 00408158     ucrt:api-ms-win-crt-runtime-l1-1-0.dll
 0002:0000015c       __imp__exit                0040815c     ucrt:api-ms-win-crt-runtime-l1-1-0.dll
 0002:00000160       __imp___exit               00408160     ucrt:api-ms-win-crt-runtime-l1-1-0.dll
 0002:00000164       __imp___initterm_e         00408164     ucrt:api-ms-win-crt-runtime-l1-1-0.dll
 0002:00000168       __imp___cexit              00408168     ucrt:api-ms-win-crt-runtime-l1-1-0.dll
 0002:0000016c       \177api-ms-win-crt-runtime-l1-1-0_NULL_THUNK_DATA 0040816c     ucrt:api-ms-win-crt-runtime-l1-1-0.dll
 0002:00000170       __imp__fclose              00408170     ucrt:api-ms-win-crt-stdio-l1-1-0.dll
 0002:00000174       __imp____stdio_common_vfwprintf 00408174     ucrt:api-ms-win-crt-stdio-l1-1-0.dll
 0002:00000178       __imp____acrt_iob_func     00408178     ucrt:api-ms-win-crt-stdio-l1-1-0.dll
 0002:0000017c       __imp____p__commode        0040817c     ucrt:api-ms-win-crt-stdio-l1-1-0.dll
 0002:00000180       __imp____stdio_common_vsprintf 00408180     ucrt:api-ms-win-crt-stdio-l1-1-0.dll
 0002:00000184       __imp__fopen               00408184     ucrt:api-ms-win-crt-stdio-l1-1-0.dll
 0002:00000188       __imp____stdio_common_vfprintf 00408188     ucrt:api-ms-win-crt-stdio-l1-1-0.dll
 0002:0000018c       __imp___set_fmode          0040818c     ucrt:api-ms-win-crt-stdio-l1-1-0.dll
 0002:00000190       __imp__fflush              00408190     ucrt:api-ms-win-crt-stdio-l1-1-0.dll
 0002:00000194       \177api-ms-win-crt-stdio-l1-1-0_NULL_THUNK_DATA 00408194     ucrt:api-ms-win-crt-stdio-l1-1-0.dll
 0002:00000198       __imp__wcscmp              00408198     ucrt:api-ms-win-crt-string-l1-1-0.dll
 0002:0000019c       __imp__strncpy             0040819c     ucrt:api-ms-win-crt-string-l1-1-0.dll
 0002:000001a0       __imp__strlen              004081a0     ucrt:api-ms-win-crt-string-l1-1-0.dll
 0002:000001a4       __imp__strcmp              004081a4     ucrt:api-ms-win-crt-string-l1-1-0.dll
 0002:000001a8       __imp__strcpy              004081a8     ucrt:api-ms-win-crt-string-l1-1-0.dll
 0002:000001ac       __imp__strncat             004081ac     ucrt:api-ms-win-crt-string-l1-1-0.dll
 0002:000001b0       \177api-ms-win-crt-string-l1-1-0_NULL_THUNK_DATA 004081b0     ucrt:api-ms-win-crt-string-l1-1-0.dll
 0002:000001b4       __imp__asctime             004081b4     ucrt:api-ms-win-crt-time-l1-1-0.dll
 0002:000001b8       __imp___time64             004081b8     ucrt:api-ms-win-crt-time-l1-1-0.dll
 0002:000001bc       __imp___localtime64        004081bc     ucrt:api-ms-win-crt-time-l1-1-0.dll
 0002:000001c0       \177api-ms-win-crt-time-l1-1-0_NULL_THUNK_DATA 004081c0     ucrt:api-ms-win-crt-time-l1-1-0.dll
 0002:000001c4       ___guard_check_icall_fptr  004081c4     MSVCRT:guard_support.obj
 0002:000001c8       ___castguard_check_failure_os_handled_fptr 004081c8     MSVCRT:guard_support.obj
 0002:000001cc       ___xc_a                    004081cc     MSVCRT:initializers.obj
 0002:000001d4       ___xc_z                    004081d4     MSVCRT:initializers.obj
 0002:000001d8       ___xi_a                    004081d8     MSVCRT:initializers.obj
 0002:000001e4       ___xi_z                    004081e4     MSVCRT:initializers.obj
 0002:000001e8       ___xp_a                    004081e8     MSVCRT:initializers.obj
 0002:000001ec       ___xp_z                    004081ec     MSVCRT:initializers.obj
 0002:000001f0       ___xt_a                    004081f0     MSVCRT:initializers.obj
 0002:000001f4       ___xt_z                    004081f4     MSVCRT:initializers.obj
 0002:00001a6c       ??_7exception@std@@6B@     00409a6c     MSVCRT:throw_bad_alloc.obj
 0002:00001a74       ??_C@_0BC@EOODALEL@Unknown?5exception@ 00409a74     MSVCRT:throw_bad_alloc.obj
 0002:00001a8c       ??_7bad_alloc@std@@6B@     00409a8c     MSVCRT:throw_bad_alloc.obj
 0002:00001a94       ??_C@_0P@GHFPNOJB@bad?5allocation@ 00409a94     MSVCRT:throw_bad_alloc.obj
 0002:00001aa8       ??_7bad_array_new_length@std@@6B@ 00409aa8     MSVCRT:throw_bad_alloc.obj
 0002:00001ab0       ??_C@_0BF@KINCDENJ@bad?5array?5new?5length@ 00409ab0     MSVCRT:throw_bad_alloc.obj
 0002:00001acc       ??_7type_info@@6B@         00409acc     MSVCRT:std_type_info_static.obj
 0002:00001ad0       __load_config_used         00409ad0     MSVCRT:loadcfg.obj
 0002:00001c00       ??_R4exception@std@@6B@    00409c00     MSVCRT:throw_bad_alloc.obj
 0002:00001c14       ??_R3exception@std@@8      00409c14     MSVCRT:throw_bad_alloc.obj
 0002:00001c24       ??_R2exception@std@@8      00409c24     MSVCRT:throw_bad_alloc.obj
 0002:00001c2c       ??_R1A@?0A@EA@exception@std@@8 00409c2c     MSVCRT:throw_bad_alloc.obj
 0002:00001c48       ??_R4bad_alloc@std@@6B@    00409c48     MSVCRT:throw_bad_alloc.obj
 0002:00001c5c       ??_R3bad_alloc@std@@8      00409c5c     MSVCRT:throw_bad_alloc.obj
 0002:00001c6c       ??_R2bad_alloc@std@@8      00409c6c     MSVCRT:throw_bad_alloc.obj
 0002:00001c78       ??_R1A@?0A@EA@bad_alloc@std@@8 00409c78     MSVCRT:throw_bad_alloc.obj
 0002:00001c94       ??_R4bad_array_new_length@std@@6B@ 00409c94     MSVCRT:throw_bad_alloc.obj
 0002:00001ca8       ??_R3bad_array_new_length@std@@8 00409ca8     MSVCRT:throw_bad_alloc.obj
 0002:00001cb8       ??_R2bad_array_new_length@std@@8 00409cb8     MSVCRT:throw_bad_alloc.obj
 0002:00001cc8       ??_R1A@?0A@EA@bad_array_new_length@std@@8 00409cc8     MSVCRT:throw_bad_alloc.obj
 0002:00001ce4       ??_R4type_info@@6B@        00409ce4     MSVCRT:std_type_info_static.obj
 0002:00001cf8       ??_R3type_info@@8          00409cf8     MSVCRT:std_type_info_static.obj
 0002:00001d08       ??_R2type_info@@8          00409d08     MSVCRT:std_type_info_static.obj
 0002:00001d10       ??_R1A@?0A@EA@type_info@@8 00409d10     MSVCRT:std_type_info_static.obj
 0002:00001d2c       ___safe_se_handler_table   00409d2c     <linker-defined>
 0002:00001d34       ___volatile_metadata       00409d34     <linker-defined>
 0002:00002110       ___rtc_iaa                 0040a110     MSVCRT:initsect.obj
 0002:00002114       ___rtc_izz                 0040a114     MSVCRT:initsect.obj
 0002:00002118       ___rtc_taa                 0040a118     MSVCRT:initsect.obj
 0002:0000211c       ___rtc_tzz                 0040a11c     MSVCRT:initsect.obj
 0002:0000216c       __TI2?AVbad_alloc@std@@    0040a16c     MSVCRT:throw_bad_alloc.obj
 0002:0000217c       __CTA2?AVbad_alloc@std@@   0040a17c     MSVCRT:throw_bad_alloc.obj
 0002:00002188       __CT??_R0?AVbad_alloc@std@@@8??0bad_alloc@std@@QAE@ABV01@@Z12 0040a188     MSVCRT:throw_bad_alloc.obj
 0002:000021a4       __CT??_R0?AVexception@std@@@8??0exception@std@@QAE@ABV01@@Z12 0040a1a4     MSVCRT:throw_bad_alloc.obj
 0002:000021c0       __TI3?AVbad_array_new_length@std@@ 0040a1c0     MSVCRT:throw_bad_alloc.obj
 0002:000021d0       __CTA3?AVbad_array_new_length@std@@ 0040a1d0     MSVCRT:throw_bad_alloc.obj
 0002:000021e0       __CT??_R0?AVbad_array_new_length@std@@@8??0bad_array_new_length@std@@QAE@ABV01@@Z12 0040a1e0     MSVCRT:throw_bad_alloc.obj
 0002:0000221c       __IMPORT_DESCRIPTOR_COMCTL32 0040a21c     comctl32:COMCTL32.dll
 0002:00002230       __IMPORT_DESCRIPTOR_GDI32  0040a230     gdi32:GDI32.dll
 0002:00002244       __IMPORT_DESCRIPTOR_USER32 0040a244     user32:USER32.dll
 0002:00002258       __IMPORT_DESCRIPTOR_KERNEL32 0040a258     kernel32:KERNEL32.dll
 0002:0000226c       __IMPORT_DESCRIPTOR_VCRUNTIME140 0040a26c     vcruntime:VCRUNTIME140.dll
 0002:00002280       __IMPORT_DESCRIPTOR_api-ms-win-crt-string-l1-1-0 0040a280     ucrt:api-ms-win-crt-string-l1-1-0.dll
 0002:00002294       __IMPORT_DESCRIPTOR_api-ms-win-crt-stdio-l1-1-0 0040a294     ucrt:api-ms-win-crt-stdio-l1-1-0.dll
 0002:000022a8       __IMPORT_DESCRIPTOR_api-ms-win-crt-environment-l1-1-0 0040a2a8     ucrt:api-ms-win-crt-environment-l1-1-0.dll
 0002:000022bc       __IMPORT_DESCRIPTOR_api-ms-win-crt-time-l1-1-0 0040a2bc     ucrt:api-ms-win-crt-time-l1-1-0.dll
 0002:000022d0       __IMPORT_DESCRIPTOR_api-ms-win-crt-heap-l1-1-0 0040a2d0     ucrt:api-ms-win-crt-heap-l1-1-0.dll
 0002:000022e4       __IMPORT_DESCRIPTOR_api-ms-win-crt-runtime-l1-1-0 0040a2e4     ucrt:api-ms-win-crt-runtime-l1-1-0.dll
 0002:000022f8       __IMPORT_DESCRIPTOR_api-ms-win-crt-math-l1-1-0 0040a2f8     ucrt:api-ms-win-crt-math-l1-1-0.dll
 0002:0000230c       __IMPORT_DESCRIPTOR_api-ms-win-crt-locale-l1-1-0 0040a30c     ucrt:api-ms-win-crt-locale-l1-1-0.dll
 0002:00002320       __NULL_IMPORT_DESCRIPTOR   0040a320     comctl32:COMCTL32.dll
 0003:00000a64       ?depth@@3HA                0040ba64     jaccesswalker.obj
 0003:00000a68       ?theJaccesswalkerClassName@@3PADA 0040ba68     jaccesswalker.obj
 0003:00000a7c       ?theAccessInfoClassName@@3PADA 0040ba7c     jaccesswalker.obj
 0003:00000ab0       ___security_cookie_complement 0040bab0     MSVCRT:gs_cookie.obj
 0003:00000ab4       ___security_cookie         0040bab4     MSVCRT:gs_cookie.obj
 0003:00000ab8       __fltused                  0040bab8     MSVCRT:fltused.obj
 0003:00000abc       ___scrt_native_dllmain_reason 0040babc     MSVCRT:utility.obj
 0003:00000ac0       ___scrt_default_matherr    0040bac0     MSVCRT:matherr.obj
 0003:00000ad0       ___isa_enabled             0040bad0     MSVCRT:cpu_disp.obj
 0003:00000ad4       ___scrt_ucrt_dll_is_in_use 0040bad4     MSVCRT:ucrt_stubs.obj
 0003:00000ad8       ??_R0?AVbad_alloc@std@@@8  0040bad8     MSVCRT:throw_bad_alloc.obj
 0003:00000af4       ??_R0?AVexception@std@@@8  0040baf4     MSVCRT:throw_bad_alloc.obj
 0003:00000b10       ??_R0?AVbad_array_new_length@std@@@8 0040bb10     MSVCRT:throw_bad_alloc.obj
 0003:00000b38       ??_R0?AVtype_info@@@8      0040bb38     MSVCRT:std_type_info_static.obj
 0003:00000b60       _theAccessBridgeInitializedFlag 0040bb60     AccessBridgeCalls.obj
 0003:00000b68       ?_OptionsStorage@?1??__local_stdio_printf_options@@9@4_KA 0040bb68     AccessBridgeDebug.obj
 0003:00000c78       ?theFromJavaHelloMsgID@@3IA 0040bc78     AccessBridgeMessages.obj
 0003:00000c7c       ?theFromWindowsHelloMsgID@@3IA 0040bc7c     AccessBridgeMessages.obj
 0003:00000c80       ?g_LogStringCallback@@3P6GXPBD@ZA 0040bc80     AccessInfo.obj
 0003:00000cc8       ?ourHwnd@@3PAUHWND__@@A    0040bcc8     jaccesswalker.obj
 0003:00000ccc       ?topLevelWindow@@3PAUHWND__@@A 0040bccc     jaccesswalker.obj
 0003:00000cd0       ?logfile@@3PAU_iobuf@@A    0040bcd0     jaccesswalker.obj
 0003:00000cd4       ?popupMenu@@3PAUHMENU__@@A 0040bcd4     jaccesswalker.obj
 0003:00000cd8       ?theJaccesswalkerWindow@@3PAUHWND__@@A 0040bcd8     jaccesswalker.obj
 0003:00000cdc       ?theTreeControlWindow@@3PAUHWND__@@A 0040bcdc     jaccesswalker.obj
 0003:00000ce0       ?theInstance@@3PAUHINSTANCE__@@A 0040bce0     jaccesswalker.obj
 0003:00000ce4       ?theJaccesswalker@@3PAVJaccesswalker@@A 0040bce4     jaccesswalker.obj
 0003:00000ce8       ?theSelectedNode@@3PAVAccessibleNode@@A 0040bce8     jaccesswalker.obj
 0003:00000cec       ?thePopupNode@@3PAVAccessibleNode@@A 0040bcec     jaccesswalker.obj
 0003:00000cf0       ?theSelectedAccessibleContext@@3PAV_jobject@@A 0040bcf0     jaccesswalker.obj
 0003:00000cf4       ?hwndTV@@3PAUHWND__@@A     0040bcf4     jaccesswalker.obj
 0003:00001014       ___scrt_current_native_startup_state 0040c014     MSVCRT:utility.obj
 0003:00001018       ___scrt_native_startup_lock 0040c018     MSVCRT:utility.obj
 0003:00001038       ?__type_info_root_node@@3U__type_info_node@@A 0040c038     MSVCRT:tncleanup.obj
 0003:00001040       ?_OptionsStorage@?1??__local_stdio_scanf_options@@9@4_KA 0040c040     MSVCRT:default_local_stdio_options.obj
 0003:00001048       ___scrt_debugger_hook_flag 0040c048     MSVCRT:utility_desktop.obj
 0003:0000104c       ___isa_available           0040c04c     MSVCRT:cpu_disp.obj
 0003:00001050       ___favor                   0040c050     MSVCRT:cpu_disp.obj
 0003:00001060       _theAccessBridge           0040c060     <common>
 0003:000011e4       _theAccessBridgeInstance   0040c1e4     <common>
 0003:000011e8       ___dyn_tls_dtor_callback   0040c1e8     <common>
 0003:000011ec       ___dyn_tls_init_callback   0040c1ec     <common>

 entry point at        0001:000062da

 Static symbols

 0000:ffff1000       .debug$S                   00400000     vcruntime:VCRUNTIME140.dll
 0000:ffff1000       .debug$S                   00400000     vcruntime:VCRUNTIME140.dll
 0000:ffff1000       .debug$S                   00400000     vcruntime:VCRUNTIME140.dll
 0000:ffff1000       .debug$S                   00400000     vcruntime:VCRUNTIME140.dll
 0000:ffff1000       .debug$S                   00400000     vcruntime:VCRUNTIME140.dll
 0000:ffff1000       .debug$S                   00400000     vcruntime:VCRUNTIME140.dll
 0000:ffff1000       .debug$S                   00400000     vcruntime:VCRUNTIME140.dll
 0000:ffff1000       .debug$S                   00400000     vcruntime:VCRUNTIME140.dll
 0000:ffff1000       .debug$S                   00400000     vcruntime:VCRUNTIME140.dll
 0000:ffff1000       .debug$S                   00400000     vcruntime:VCRUNTIME140.dll
 0000:ffff1000       .debug$S                   00400000     ucrt:api-ms-win-crt-environment-l1-1-0.dll
 0000:ffff1000       .debug$S                   00400000     ucrt:api-ms-win-crt-heap-l1-1-0.dll
 0000:ffff1000       .debug$S                   00400000     ucrt:api-ms-win-crt-heap-l1-1-0.dll
 0000:ffff1000       .debug$S                   00400000     ucrt:api-ms-win-crt-heap-l1-1-0.dll
 0000:ffff1000       .debug$S                   00400000     ucrt:api-ms-win-crt-heap-l1-1-0.dll
 0000:ffff1000       .debug$S                   00400000     ucrt:api-ms-win-crt-locale-l1-1-0.dll
 0000:ffff1000       .debug$S                   00400000     ucrt:api-ms-win-crt-math-l1-1-0.dll
 0000:ffff1000       .debug$S                   00400000     ucrt:api-ms-win-crt-runtime-l1-1-0.dll
 0000:ffff1000       .debug$S                   00400000     ucrt:api-ms-win-crt-runtime-l1-1-0.dll
 0000:ffff1000       .debug$S                   00400000     ucrt:api-ms-win-crt-runtime-l1-1-0.dll
 0000:ffff1000       .debug$S                   00400000     ucrt:api-ms-win-crt-runtime-l1-1-0.dll
 0000:ffff1000       .debug$S                   00400000     ucrt:api-ms-win-crt-runtime-l1-1-0.dll
 0000:ffff1000       .debug$S                   00400000     ucrt:api-ms-win-crt-runtime-l1-1-0.dll
 0000:ffff1000       .debug$S                   00400000     ucrt:api-ms-win-crt-runtime-l1-1-0.dll
 0000:ffff1000       .debug$S                   00400000     ucrt:api-ms-win-crt-runtime-l1-1-0.dll
 0000:ffff1000       .debug$S                   00400000     ucrt:api-ms-win-crt-runtime-l1-1-0.dll
 0000:ffff1000       .debug$S                   00400000     ucrt:api-ms-win-crt-runtime-l1-1-0.dll
 0000:ffff1000       .debug$S                   00400000     ucrt:api-ms-win-crt-runtime-l1-1-0.dll
 0000:ffff1000       .debug$S                   00400000     ucrt:api-ms-win-crt-runtime-l1-1-0.dll
 0000:ffff1000       .debug$S                   00400000     ucrt:api-ms-win-crt-runtime-l1-1-0.dll
 0000:ffff1000       .debug$S                   00400000     ucrt:api-ms-win-crt-runtime-l1-1-0.dll
 0000:ffff1000       .debug$S                   00400000     ucrt:api-ms-win-crt-runtime-l1-1-0.dll
 0000:ffff1000       .debug$S                   00400000     ucrt:api-ms-win-crt-runtime-l1-1-0.dll
 0000:ffff1000       .debug$S                   00400000     ucrt:api-ms-win-crt-runtime-l1-1-0.dll
 0000:ffff1000       .debug$S                   00400000     ucrt:api-ms-win-crt-runtime-l1-1-0.dll
 0000:ffff1000       .debug$S                   00400000     ucrt:api-ms-win-crt-runtime-l1-1-0.dll
 0000:ffff1000       .debug$S                   00400000     ucrt:api-ms-win-crt-runtime-l1-1-0.dll
 0000:ffff1000       .debug$S                   00400000     ucrt:api-ms-win-crt-stdio-l1-1-0.dll
 0000:ffff1000       .debug$S                   00400000     ucrt:api-ms-win-crt-stdio-l1-1-0.dll
 0000:ffff1000       .debug$S                   00400000     ucrt:api-ms-win-crt-stdio-l1-1-0.dll
 0000:ffff1000       .debug$S                   00400000     ucrt:api-ms-win-crt-stdio-l1-1-0.dll
 0000:ffff1000       .debug$S                   00400000     ucrt:api-ms-win-crt-stdio-l1-1-0.dll
 0000:ffff1000       .debug$S                   00400000     ucrt:api-ms-win-crt-stdio-l1-1-0.dll
 0000:ffff1000       .debug$S                   00400000     ucrt:api-ms-win-crt-stdio-l1-1-0.dll
 0000:ffff1000       .debug$S                   00400000     ucrt:api-ms-win-crt-stdio-l1-1-0.dll
 0000:ffff1000       .debug$S                   00400000     ucrt:api-ms-win-crt-stdio-l1-1-0.dll
 0000:ffff1000       .debug$S                   00400000     ucrt:api-ms-win-crt-string-l1-1-0.dll
 0000:ffff1000       .debug$S                   00400000     ucrt:api-ms-win-crt-string-l1-1-0.dll
 0000:ffff1000       .debug$S                   00400000     ucrt:api-ms-win-crt-string-l1-1-0.dll
 0000:ffff1000       .debug$S                   00400000     ucrt:api-ms-win-crt-string-l1-1-0.dll
 0000:ffff1000       .debug$S                   00400000     ucrt:api-ms-win-crt-string-l1-1-0.dll
 0000:ffff1000       .debug$S                   00400000     ucrt:api-ms-win-crt-string-l1-1-0.dll
 0000:ffff1000       .debug$S                   00400000     ucrt:api-ms-win-crt-time-l1-1-0.dll
 0000:ffff1000       .debug$S                   00400000     ucrt:api-ms-win-crt-time-l1-1-0.dll
 0000:ffff1000       .debug$S                   00400000     ucrt:api-ms-win-crt-time-l1-1-0.dll
 0000:ffff1000       .debug$S                   00400000     comctl32:COMCTL32.dll
 0000:ffff1000       .debug$S                   00400000     gdi32:GDI32.dll
 0000:ffff1000       .debug$S                   00400000     kernel32:KERNEL32.dll
 0000:ffff1000       .debug$S                   00400000     kernel32:KERNEL32.dll
 0000:ffff1000       .debug$S                   00400000     kernel32:KERNEL32.dll
 0000:ffff1000       .debug$S                   00400000     kernel32:KERNEL32.dll
 0000:ffff1000       .debug$S                   00400000     kernel32:KERNEL32.dll
 0000:ffff1000       .debug$S                   00400000     kernel32:KERNEL32.dll
 0000:ffff1000       .debug$S                   00400000     kernel32:KERNEL32.dll
 0000:ffff1000       .debug$S                   00400000     kernel32:KERNEL32.dll
 0000:ffff1000       .debug$S                   00400000     kernel32:KERNEL32.dll
 0000:ffff1000       .debug$S                   00400000     kernel32:KERNEL32.dll
 0000:ffff1000       .debug$S                   00400000     kernel32:KERNEL32.dll
 0000:ffff1000       .debug$S                   00400000     kernel32:KERNEL32.dll
 0000:ffff1000       .debug$S                   00400000     kernel32:KERNEL32.dll
 0000:ffff1000       .debug$S                   00400000     kernel32:KERNEL32.dll
 0000:ffff1000       .debug$S                   00400000     kernel32:KERNEL32.dll
 0000:ffff1000       .debug$S                   00400000     kernel32:KERNEL32.dll
 0000:ffff1000       .debug$S                   00400000     kernel32:KERNEL32.dll
 0000:ffff1000       .debug$S                   00400000     kernel32:KERNEL32.dll
 0000:ffff1000       .debug$S                   00400000     kernel32:KERNEL32.dll
 0000:ffff1000       .debug$S                   00400000     user32:USER32.dll
 0000:ffff1000       .debug$S                   00400000     user32:USER32.dll
 0000:ffff1000       .debug$S                   00400000     user32:USER32.dll
 0000:ffff1000       .debug$S                   00400000     user32:USER32.dll
 0000:ffff1000       .debug$S                   00400000     user32:USER32.dll
 0000:ffff1000       .debug$S                   00400000     user32:USER32.dll
 0000:ffff1000       .debug$S                   00400000     user32:USER32.dll
 0000:ffff1000       .debug$S                   00400000     user32:USER32.dll
 0000:ffff1000       .debug$S                   00400000     user32:USER32.dll
 0000:ffff1000       .debug$S                   00400000     user32:USER32.dll
 0000:ffff1000       .debug$S                   00400000     user32:USER32.dll
 0000:ffff1000       .debug$S                   00400000     user32:USER32.dll
 0000:ffff1000       .debug$S                   00400000     user32:USER32.dll
 0000:ffff1000       .debug$S                   00400000     user32:USER32.dll
 0000:ffff1000       .debug$S                   00400000     user32:USER32.dll
 0000:ffff1000       .debug$S                   00400000     user32:USER32.dll
 0000:ffff1000       .debug$S                   00400000     user32:USER32.dll
 0000:ffff1000       .debug$S                   00400000     user32:USER32.dll
 0000:ffff1000       .debug$S                   00400000     user32:USER32.dll
 0000:ffff1000       .debug$S                   00400000     user32:USER32.dll
 0000:ffff1000       .debug$S                   00400000     user32:USER32.dll
 0000:ffff1000       .debug$S                   00400000     user32:USER32.dll
 0000:ffff1000       .debug$S                   00400000     user32:USER32.dll
 0000:ffff1000       .debug$S                   00400000     user32:USER32.dll
 0000:ffff1000       .debug$S                   00400000     user32:USER32.dll
 0000:ffff1000       .debug$S                   00400000     user32:USER32.dll
 0000:ffff1000       .debug$S                   00400000     user32:USER32.dll
 0000:ffff1000       .debug$S                   00400000     user32:USER32.dll
 0001:000047b0       _localtime                 004057b0 f   AccessInfo.obj
 0001:000047d0       _time                      004057d0 f   AccessInfo.obj
 0001:0000530c       $LN26                      0040630c     jaccesswalker.obj
 0001:00005320       $LN25                      00406320     jaccesswalker.obj
 0001:00005fb0       $$000000                   00406fb0     MSVCRT:ulldiv.obj
 0001:00005fd2       L1                         00406fd2     MSVCRT:ulldiv.obj
 0001:00005fe0       L3                         00406fe0     MSVCRT:ulldiv.obj
 0001:0000600e       L4                         0040700e     MSVCRT:ulldiv.obj
 0001:0000600f       L5                         0040700f     MSVCRT:ulldiv.obj
 0001:00006013       L2                         00407013     MSVCRT:ulldiv.obj
 0001:00006030       $$000000                   00407030     MSVCRT:chkstk.obj
 0001:00006044       cs10                       00407044     MSVCRT:chkstk.obj
 0001:00006052       cs20                       00407052     MSVCRT:chkstk.obj
 0001:00006099       ?pre_c_initialization@@YAHXZ 00407099 f   MSVCRT:exe_winmain.obj
 0001:00006144       ?post_pgo_initialization@@YAHXZ 00407144 f   MSVCRT:exe_winmain.obj
 0001:0000614c       ?pre_cpp_initialization@@YAXXZ 0040714c f   MSVCRT:exe_winmain.obj
 0001:0000615e       ?__scrt_common_main_seh@@YAHXZ 0040715e f   MSVCRT:exe_winmain.obj
 0001:00006400       ?find_pe_section@@YAPAU_IMAGE_SECTION_HEADER@@QAEI@Z 00407400 f   MSVCRT:utility.obj
 0001:00006651       ___get_entropy             00407651 f   MSVCRT:gs_support.obj
 0001:000069c0       $$000000                   004079c0     MSVCRT:sehprolg4.obj
 0001:00006d90       __unwindfunclet$?addComponentNodes@Jaccesswalker@@QAEXJPAV_jobject@@PAVAccessibleNode@@PAUHWND__@@PAU_TREEITEM@@2@Z$0 00407d90 f   jaccesswalker.obj
 0001:00006daa       __ehhandler$?addComponentNodes@Jaccesswalker@@QAEXJPAV_jobject@@PAVAccessibleNode@@PAUHWND__@@PAU_TREEITEM@@2@Z 00407daa f   jaccesswalker.obj
 0002:000001d0       ?pre_cpp_initializer@@3P6AXXZA 004081d0     MSVCRT:exe_winmain.obj
 0002:000001dc       ?pre_c_initializer@@3P6AHXZA 004081dc     MSVCRT:exe_winmain.obj
 0002:000001e0       ?post_pgo_initializer@@3P6AHXZA 004081e0     MSVCRT:exe_winmain.obj
 0002:000001f8       $SG44893                   004081f8     AccessBridgeDebug.obj
 0002:00000214       $SG44895                   00408214     AccessBridgeDebug.obj
 0002:0000021c       $SG44896                   0040821c     AccessBridgeDebug.obj
 0002:00000220       $SG44898                   00408220     AccessBridgeDebug.obj
 0002:00000228       $SG44899                   00408228     AccessBridgeDebug.obj
 0002:00000240       $SG44926                   00408240     AccessBridgeDebug.obj
 0002:0000025c       $SG44927                   0040825c     AccessBridgeDebug.obj
 0002:00000268       $SG44929                   00408268     AccessBridgeDebug.obj
 0002:0000026c       $SG44971                   0040826c     AccessBridgeDebug.obj
 0002:00000274       $SG44972                   00408274     AccessBridgeDebug.obj
 0002:00000278       $SG44988                   00408278     AccessBridgeDebug.obj
 0002:00000280       $SG44989                   00408280     AccessBridgeDebug.obj
 0002:00000284       $SG45031                   00408284     AccessBridgeDebug.obj
 0002:0000028c       $SG45032                   0040828c     AccessBridgeDebug.obj
 0002:00000290       $SG45048                   00408290     AccessBridgeDebug.obj
 0002:00000298       $SG45049                   00408298     AccessBridgeDebug.obj
 0002:0000029c       $SG39804                   0040829c     AccessBridgeMessages.obj
 0002:000002b8       $SG39805                   004082b8     AccessBridgeMessages.obj
 0002:000002d8       $SG49224                   004082d8     AccessInfo.obj
 0002:000002dc       $SG49226                   004082dc     AccessInfo.obj
 0002:000002e0       $SG49229                   004082e0     AccessInfo.obj
 0002:000002ec       $SG49274                   004082ec     AccessInfo.obj
 0002:00000318       $SG49275                   00408318     AccessInfo.obj
 0002:0000031c       $SG49276                   0040831c     AccessInfo.obj
 0002:00000320       $SG49294                   00408320     AccessInfo.obj
 0002:00000324       $SG49436                   00408324     AccessInfo.obj
 0002:0000034c       $SG49437                   0040834c     AccessInfo.obj
 0002:00000364       $SG49438                   00408364     AccessInfo.obj
 0002:0000038c       $SG49439                   0040838c     AccessInfo.obj
 0002:000003b8       $SG49440                   004083b8     AccessInfo.obj
 0002:000003e4       $SG49441                   004083e4     AccessInfo.obj
 0002:00000414       $SG49445                   00408414     AccessInfo.obj
 0002:00000440       $SG49446                   00408440     AccessInfo.obj
 0002:00000464       $SG49449                   00408464     AccessInfo.obj
 0002:00000480       $SG49450                   00408480     AccessInfo.obj
 0002:00000484       $SG49451                   00408484     AccessInfo.obj
 0002:00000498       $SG49454                   00408498     AccessInfo.obj
 0002:000004bc       $SG49455                   004084bc     AccessInfo.obj
 0002:000004d8       $SG49456                   004084d8     AccessInfo.obj
 0002:000004f0       $SG49457                   004084f0     AccessInfo.obj
 0002:00000504       $SG49458                   00408504     AccessInfo.obj
 0002:00000528       $SG49459                   00408528     AccessInfo.obj
 0002:0000053c       $SG49460                   0040853c     AccessInfo.obj
 0002:00000560       $SG49461                   00408560     AccessInfo.obj
 0002:0000057c       $SG49462                   0040857c     AccessInfo.obj
 0002:00000598       $SG49463                   00408598     AccessInfo.obj
 0002:000005c4       $SG49466                   004085c4     AccessInfo.obj
 0002:000005e8       $SG49469                   004085e8     AccessInfo.obj
 0002:00000628       $SG49472                   00408628     AccessInfo.obj
 0002:0000064c       $SG49473                   0040864c     AccessInfo.obj
 0002:00000670       $SG49474                   00408670     AccessInfo.obj
 0002:00000694       $SG49477                   00408694     AccessInfo.obj
 0002:000006a4       $SG49480                   004086a4     AccessInfo.obj
 0002:000006d8       $SG49481                   004086d8     AccessInfo.obj
 0002:000006f0       $SG49484                   004086f0     AccessInfo.obj
 0002:00000714       $SG49485                   00408714     AccessInfo.obj
 0002:00000734       $SG49486                   00408734     AccessInfo.obj
 0002:0000074c       $SG49489                   0040874c     AccessInfo.obj
 0002:00000774       $SG49490                   00408774     AccessInfo.obj
 0002:0000079c       $SG49494                   0040879c     AccessInfo.obj
 0002:000007c0       $SG49498                   004087c0     AccessInfo.obj
 0002:000007e4       $SG49499                   004087e4     AccessInfo.obj
 0002:00000804       $SG49500                   00408804     AccessInfo.obj
 0002:00000824       $SG49502                   00408824     AccessInfo.obj
 0002:0000084c       $SG49504                   0040884c     AccessInfo.obj
 0002:00000868       $SG49507                   00408868     AccessInfo.obj
 0002:000008ac       $SG49510                   004088ac     AccessInfo.obj
 0002:000008e8       $SG49513                   004088e8     AccessInfo.obj
 0002:0000090c       $SG49514                   0040890c     AccessInfo.obj
 0002:0000092c       $SG49515                   0040892c     AccessInfo.obj
 0002:0000094c       $SG49516                   0040894c     AccessInfo.obj
 0002:00000978       $SG49518                   00408978     AccessInfo.obj
 0002:00000998       $SG49519                   00408998     AccessInfo.obj
 0002:000009bc       $SG49520                   004089bc     AccessInfo.obj
 0002:000009e0       $SG49521                   004089e0     AccessInfo.obj
 0002:00000a04       $SG49523                   00408a04     AccessInfo.obj
 0002:00000a20       $SG49524                   00408a20     AccessInfo.obj
 0002:00000a3c       $SG49525                   00408a3c     AccessInfo.obj
 0002:00000a5c       $SG49526                   00408a5c     AccessInfo.obj
 0002:00000a78       $SG49527                   00408a78     AccessInfo.obj
 0002:00000a90       $SG49529                   00408a90     AccessInfo.obj
 0002:00000aac       $SG49530                   00408aac     AccessInfo.obj
 0002:00000acc       $SG49531                   00408acc     AccessInfo.obj
 0002:00000ae8       $SG49534                   00408ae8     AccessInfo.obj
 0002:00000b0c       $SG49536                   00408b0c     AccessInfo.obj
 0002:00000b34       $SG49537                   00408b34     AccessInfo.obj
 0002:00000b54       $SG49538                   00408b54     AccessInfo.obj
 0002:00000b70       $SG49539                   00408b70     AccessInfo.obj
 0002:00000b94       $SG49542                   00408b94     AccessInfo.obj
 0002:00000bc0       $SG49545                   00408bc0     AccessInfo.obj
 0002:00000be4       $SG49546                   00408be4     AccessInfo.obj
 0002:00000c04       $SG49547                   00408c04     AccessInfo.obj
 0002:00000c24       $SG49549                   00408c24     AccessInfo.obj
 0002:00000c48       $SG49551                   00408c48     AccessInfo.obj
 0002:00000c64       $SG49553                   00408c64     AccessInfo.obj
 0002:00000c80       $SG49555                   00408c80     AccessInfo.obj
 0002:00000c9c       $SG49559                   00408c9c     AccessInfo.obj
 0002:00000cc4       $SG49560                   00408cc4     AccessInfo.obj
 0002:00000ce0       $SG49561                   00408ce0     AccessInfo.obj
 0002:00000d04       $SG49562                   00408d04     AccessInfo.obj
 0002:00000d28       $SG49563                   00408d28     AccessInfo.obj
 0002:00000d4c       $SG49564                   00408d4c     AccessInfo.obj
 0002:00000d68       $SG49565                   00408d68     AccessInfo.obj
 0002:00000d88       $SG49568                   00408d88     AccessInfo.obj
 0002:00000db4       $SG49569                   00408db4     AccessInfo.obj
 0002:00000de0       $SG49570                   00408de0     AccessInfo.obj
 0002:00000df4       $SG49571                   00408df4     AccessInfo.obj
 0002:00000e0c       $SG49572                   00408e0c     AccessInfo.obj
 0002:00000e28       $SG49573                   00408e28     AccessInfo.obj
 0002:00000e40       $SG49576                   00408e40     AccessInfo.obj
 0002:00000e84       $SG49579                   00408e84     AccessInfo.obj
 0002:00000ea8       $SG49580                   00408ea8     AccessInfo.obj
 0002:00000ebc       $SG49581                   00408ebc     AccessInfo.obj
 0002:00000ed0       $SG49584                   00408ed0     AccessInfo.obj
 0002:00000f00       $SG49585                   00408f00     AccessInfo.obj
 0002:00000f28       $SG49586                   00408f28     AccessInfo.obj
 0002:00000f4c       $SG49587                   00408f4c     AccessInfo.obj
 0002:00000f74       $SG49588                   00408f74     AccessInfo.obj
 0002:00000f94       $SG49591                   00408f94     AccessInfo.obj
 0002:00000fc8       $SG49592                   00408fc8     AccessInfo.obj
 0002:00000fe0       $SG49593                   00408fe0     AccessInfo.obj
 0002:00000fe4       $SG49596                   00408fe4     AccessInfo.obj
 0002:00001010       $SG49597                   00409010     AccessInfo.obj
 0002:00001034       $SG49598                   00409034     AccessInfo.obj
 0002:00001048       $SG49599                   00409048     AccessInfo.obj
 0002:00001060       $SG49600                   00409060     AccessInfo.obj
 0002:0000107c       $SG49601                   0040907c     AccessInfo.obj
 0002:00001094       $SG49604                   00409094     AccessInfo.obj
 0002:000010c0       $SG49607                   004090c0     AccessInfo.obj
 0002:000010e4       $SG49608                   004090e4     AccessInfo.obj
 0002:000010f8       $SG49609                   004090f8     AccessInfo.obj
 0002:0000110c       $SG49611                   0040910c     AccessInfo.obj
 0002:00001130       $SG49613                   00409130     AccessInfo.obj
 0002:00001158       $SG49614                   00409158     AccessInfo.obj
 0002:00001178       $SG49615                   00409178     AccessInfo.obj
 0002:00001190       $SG49617                   00409190     AccessInfo.obj
 0002:000011b4       $SG49618                   004091b4     AccessInfo.obj
 0002:000011d4       $SG49619                   004091d4     AccessInfo.obj
 0002:000011f0       $SG49620                   004091f0     AccessInfo.obj
 0002:00001214       $SG49622                   00409214     AccessInfo.obj
 0002:00001250       $SG49625                   00409250     AccessInfo.obj
 0002:00001270       $SG49627                   00409270     AccessInfo.obj
 0002:0000128c       $SG49628                   0040928c     AccessInfo.obj
 0002:000012a4       $SG49629                   004092a4     AccessInfo.obj
 0002:000012c0       $SG49631                   004092c0     AccessInfo.obj
 0002:000012c8       $SG49632                   004092c8     AccessInfo.obj
 0002:000012d4       $SG49633                   004092d4     AccessInfo.obj
 0002:000012f4       $SG49634                   004092f4     AccessInfo.obj
 0002:000012fc       $SG49635                   004092fc     AccessInfo.obj
 0002:00001308       $SG49636                   00409308     AccessInfo.obj
 0002:00001310       $SG49637                   00409310     AccessInfo.obj
 0002:0000131c       $SG49638                   0040931c     AccessInfo.obj
 0002:0000132c       $SG49639                   0040932c     AccessInfo.obj
 0002:00001334       $SG49640                   00409334     AccessInfo.obj
 0002:00001344       $SG49641                   00409344     AccessInfo.obj
 0002:00001358       $SG49642                   00409358     AccessInfo.obj
 0002:00001360       $SG49643                   00409360     AccessInfo.obj
 0002:0000136c       $SG49644                   0040936c     AccessInfo.obj
 0002:0000137c       $SG49645                   0040937c     AccessInfo.obj
 0002:00001384       $SG49646                   00409384     AccessInfo.obj
 0002:00001390       $SG49647                   00409390     AccessInfo.obj
 0002:000013a0       $SG49648                   004093a0     AccessInfo.obj
 0002:000013a8       $SG49649                   004093a8     AccessInfo.obj
 0002:000013cc       $SG49650                   004093cc     AccessInfo.obj
 0002:000013f0       $SG49651                   004093f0     AccessInfo.obj
 0002:0000140c       $SG49652                   0040940c     AccessInfo.obj
 0002:00001428       $SG49653                   00409428     AccessInfo.obj
 0002:0000144c       $SG49654                   0040944c     AccessInfo.obj
 0002:00001468       $SG49655                   00409468     AccessInfo.obj
 0002:00001484       $SG49656                   00409484     AccessInfo.obj
 0002:000014a0       $SG49657                   004094a0     AccessInfo.obj
 0002:000014bc       $SG49658                   004094bc     AccessInfo.obj
 0002:000014d8       $SG49659                   004094d8     AccessInfo.obj
 0002:00001500       $SG49662                   00409500     AccessInfo.obj
 0002:00001520       $SG49663                   00409520     AccessInfo.obj
 0002:0000154c       $SG49664                   0040954c     AccessInfo.obj
 0002:00001568       $SG49666                   00409568     AccessInfo.obj
 0002:000015a0       $SG49668                   004095a0     AccessInfo.obj
 0002:000015dc       $SG49671                   004095dc     AccessInfo.obj
 0002:000015fc       $SG49673                   004095fc     AccessInfo.obj
 0002:00001618       $SG49674                   00409618     AccessInfo.obj
 0002:00001630       $SG49675                   00409630     AccessInfo.obj
 0002:0000164c       $SG49677                   0040964c     AccessInfo.obj
 0002:00001654       $SG49678                   00409654     AccessInfo.obj
 0002:00001660       $SG49679                   00409660     AccessInfo.obj
 0002:00001680       $SG49680                   00409680     AccessInfo.obj
 0002:00001688       $SG49681                   00409688     AccessInfo.obj
 0002:00001694       $SG49682                   00409694     AccessInfo.obj
 0002:0000169c       $SG49683                   0040969c     AccessInfo.obj
 0002:000016a8       $SG49684                   004096a8     AccessInfo.obj
 0002:000016b8       $SG49685                   004096b8     AccessInfo.obj
 0002:000016c0       $SG49686                   004096c0     AccessInfo.obj
 0002:000016d0       $SG49687                   004096d0     AccessInfo.obj
 0002:000016e4       $SG49688                   004096e4     AccessInfo.obj
 0002:000016ec       $SG49689                   004096ec     AccessInfo.obj
 0002:000016f8       $SG49690                   004096f8     AccessInfo.obj
 0002:00001708       $SG49691                   00409708     AccessInfo.obj
 0002:00001710       $SG49692                   00409710     AccessInfo.obj
 0002:0000171c       $SG49693                   0040971c     AccessInfo.obj
 0002:0000172c       $SG49694                   0040972c     AccessInfo.obj
 0002:00001734       $SG49695                   00409734     AccessInfo.obj
 0002:00001758       $SG49696                   00409758     AccessInfo.obj
 0002:0000177c       $SG49697                   0040977c     AccessInfo.obj
 0002:00001798       $SG49698                   00409798     AccessInfo.obj
 0002:000017b4       $SG49699                   004097b4     AccessInfo.obj
 0002:000017d8       $SG49700                   004097d8     AccessInfo.obj
 0002:000017f4       $SG49701                   004097f4     AccessInfo.obj
 0002:00001810       $SG49702                   00409810     AccessInfo.obj
 0002:0000182c       $SG49703                   0040982c     AccessInfo.obj
 0002:00001848       $SG49704                   00409848     AccessInfo.obj
 0002:00001864       $SG49705                   00409864     AccessInfo.obj
 0002:0000188c       $SG49708                   0040988c     AccessInfo.obj
 0002:000018ac       $SG49709                   004098ac     AccessInfo.obj
 0002:000018d8       $SG57371                   004098d8     jaccesswalker.obj
 0002:000018f4       $SG57373                   004098f4     jaccesswalker.obj
 0002:0000190d       $SG57114                   0040990d     jaccesswalker.obj
 0002:0000190e       $SG57188                   0040990e     jaccesswalker.obj
 0002:0000190f       $SG57291                   0040990f     jaccesswalker.obj
 0002:00001910       $SG57066                   00409910     jaccesswalker.obj
 0002:00001914       $SG57067                   00409914     jaccesswalker.obj
 0002:00001928       $SG57068                   00409928     jaccesswalker.obj
 0002:00001948       $SG57154                   00409948     jaccesswalker.obj
 0002:00001954       $SG57189                   00409954     jaccesswalker.obj
 0002:0000195c       $SG57217                   0040995c     jaccesswalker.obj
 0002:00001964       $SG57218                   00409964     jaccesswalker.obj
 0002:0000197c       $SG57241                   0040997c     jaccesswalker.obj
 0002:00001988       $SG57248                   00409988     jaccesswalker.obj
 0002:00001994       $SG57252                   00409994     jaccesswalker.obj
 0002:000019a0       $SG57254                   004099a0     jaccesswalker.obj
 0002:000019ac       $SG57257                   004099ac     jaccesswalker.obj
 0002:000019b8       $SG57259                   004099b8     jaccesswalker.obj
 0002:000019c8       $SG57261                   004099c8     jaccesswalker.obj
 0002:000019d4       $SG57266                   004099d4     jaccesswalker.obj
 0002:000019e0       $SG57268                   004099e0     jaccesswalker.obj
 0002:000019ec       $SG57271                   004099ec     jaccesswalker.obj
 0002:000019f8       $SG57292                   004099f8     jaccesswalker.obj
 0002:00001a08       $SG57338                   00409a08     jaccesswalker.obj
 0002:00001a0c       $SG57339                   00409a0c     jaccesswalker.obj
 0002:00001a10       $SG57340                   00409a10     jaccesswalker.obj
 0002:00001a20       $SG57341                   00409a20     jaccesswalker.obj
 0002:00001a60       _GS_ExceptionPointers      00409a60     MSVCRT:gs_report.obj
 0002:00002120       __unwindtable$?addComponentNodes@Jaccesswalker@@QAEXJPAV_jobject@@PAVAccessibleNode@@PAUHWND__@@PAU_TREEITEM@@2@Z 0040a120     jaccesswalker.obj
 0002:00002128       __ehfuncinfo$?addComponentNodes@Jaccesswalker@@QAEXJPAV_jobject@@PAVAccessibleNode@@PAUHWND__@@PAU_TREEITEM@@2@Z 0040a128     jaccesswalker.obj
 0002:00002150       __sehtable$?__scrt_common_main_seh@@YAHXZ 0040a150     MSVCRT:exe_winmain.obj
 0002:00002200       __sehtable$___scrt_is_nonwritable_in_current_image 0040a200     MSVCRT:utility.obj
 0002:00002510       .idata$6                   0040a510     comctl32:COMCTL32.dll
 0002:00002530       .idata$6                   0040a530     gdi32:GDI32.dll
 0002:00002704       .idata$6                   0040a704     user32:USER32.dll
 0002:0000289c       .idata$6                   0040a89c     kernel32:KERNEL32.dll
 0002:0000296a       .idata$6                   0040a96a     vcruntime:VCRUNTIME140.dll
 0002:00002c2a       .idata$6                   0040ac2a     ucrt:api-ms-win-crt-string-l1-1-0.dll
 0002:00002c4c       .idata$6                   0040ac4c     ucrt:api-ms-win-crt-stdio-l1-1-0.dll
 0002:00002c6c       .idata$6                   0040ac6c     ucrt:api-ms-win-crt-environment-l1-1-0.dll
 0002:00002c92       .idata$6                   0040ac92     ucrt:api-ms-win-crt-time-l1-1-0.dll
 0002:00002cb2       .idata$6                   0040acb2     ucrt:api-ms-win-crt-heap-l1-1-0.dll
 0002:00002cd2       .idata$6                   0040acd2     ucrt:api-ms-win-crt-runtime-l1-1-0.dll
 0002:00002cf4       .idata$6                   0040acf4     ucrt:api-ms-win-crt-math-l1-1-0.dll
 0002:00002d14       .idata$6                   0040ad14     ucrt:api-ms-win-crt-locale-l1-1-0.dll
 0003:00000000       $SG37182                   0040b000     AccessBridgeCalls.obj
 0003:00000014       $SG37186                   0040b014     AccessBridgeCalls.obj
 0003:00000020       $SG37188                   0040b020     AccessBridgeCalls.obj
 0003:00000034       $SG37190                   0040b034     AccessBridgeCalls.obj
 0003:00000048       $SG37192                   0040b048     AccessBridgeCalls.obj
 0003:00000058       $SG37194                   0040b058     AccessBridgeCalls.obj
 0003:0000006c       $SG37196                   0040b06c     AccessBridgeCalls.obj
 0003:00000080       $SG37198                   0040b080     AccessBridgeCalls.obj
 0003:00000094       $SG37200                   0040b094     AccessBridgeCalls.obj
 0003:000000a8       $SG37202                   0040b0a8     AccessBridgeCalls.obj
 0003:000000bc       $SG37204                   0040b0bc     AccessBridgeCalls.obj
 0003:000000d0       $SG37206                   0040b0d0     AccessBridgeCalls.obj
 0003:000000e4       $SG37208                   0040b0e4     AccessBridgeCalls.obj
 0003:000000f8       $SG37210                   0040b0f8     AccessBridgeCalls.obj
 0003:0000010c       $SG37212                   0040b10c     AccessBridgeCalls.obj
 0003:00000124       $SG37214                   0040b124     AccessBridgeCalls.obj
 0003:00000148       $SG37216                   0040b148     AccessBridgeCalls.obj
 0003:00000168       $SG37218                   0040b168     AccessBridgeCalls.obj
 0003:00000180       $SG37220                   0040b180     AccessBridgeCalls.obj
 0003:000001a0       $SG37222                   0040b1a0     AccessBridgeCalls.obj
 0003:000001bc       $SG37224                   0040b1bc     AccessBridgeCalls.obj
 0003:000001d8       $SG37226                   0040b1d8     AccessBridgeCalls.obj
 0003:000001f8       $SG37228                   0040b1f8     AccessBridgeCalls.obj
 0003:00000210       $SG37230                   0040b210     AccessBridgeCalls.obj
 0003:0000022c       $SG37232                   0040b22c     AccessBridgeCalls.obj
 0003:0000024c       $SG37234                   0040b24c     AccessBridgeCalls.obj
 0003:00000268       $SG37236                   0040b268     AccessBridgeCalls.obj
 0003:0000028c       $SG37238                   0040b28c     AccessBridgeCalls.obj
 0003:000002ac       $SG37240                   0040b2ac     AccessBridgeCalls.obj
 0003:000002c0       $SG37242                   0040b2c0     AccessBridgeCalls.obj
 0003:000002d0       $SG37244                   0040b2d0     AccessBridgeCalls.obj
 0003:000002e0       $SG37246                   0040b2e0     AccessBridgeCalls.obj
 0003:000002f0       $SG37248                   0040b2f0     AccessBridgeCalls.obj
 0003:00000310       $SG37250                   0040b310     AccessBridgeCalls.obj
 0003:00000330       $SG37252                   0040b330     AccessBridgeCalls.obj
 0003:00000348       $SG37254                   0040b348     AccessBridgeCalls.obj
 0003:00000368       $SG37256                   0040b368     AccessBridgeCalls.obj
 0003:00000384       $SG37258                   0040b384     AccessBridgeCalls.obj
 0003:000003a4       $SG37260                   0040b3a4     AccessBridgeCalls.obj
 0003:000003c4       $SG37262                   0040b3c4     AccessBridgeCalls.obj
 0003:000003dc       $SG37264                   0040b3dc     AccessBridgeCalls.obj
 0003:000003f8       $SG37266                   0040b3f8     AccessBridgeCalls.obj
 0003:00000414       $SG37268                   0040b414     AccessBridgeCalls.obj
 0003:00000434       $SG37270                   0040b434     AccessBridgeCalls.obj
 0003:00000458       $SG37272                   0040b458     AccessBridgeCalls.obj
 0003:0000047c       $SG37274                   0040b47c     AccessBridgeCalls.obj
 0003:000004a0       $SG37276                   0040b4a0     AccessBridgeCalls.obj
 0003:000004c0       $SG37278                   0040b4c0     AccessBridgeCalls.obj
 0003:000004e0       $SG37280                   0040b4e0     AccessBridgeCalls.obj
 0003:00000508       $SG37282                   0040b508     AccessBridgeCalls.obj
 0003:00000528       $SG37284                   0040b528     AccessBridgeCalls.obj
 0003:0000054c       $SG37286                   0040b54c     AccessBridgeCalls.obj
 0003:00000564       $SG37288                   0040b564     AccessBridgeCalls.obj
 0003:00000580       $SG37290                   0040b580     AccessBridgeCalls.obj
 0003:00000598       $SG37292                   0040b598     AccessBridgeCalls.obj
 0003:000005b4       $SG37294                   0040b5b4     AccessBridgeCalls.obj
 0003:000005cc       $SG37296                   0040b5cc     AccessBridgeCalls.obj
 0003:000005e8       $SG37298                   0040b5e8     AccessBridgeCalls.obj
 0003:00000604       $SG37300                   0040b604     AccessBridgeCalls.obj
 0003:00000620       $SG37302                   0040b620     AccessBridgeCalls.obj
 0003:00000640       $SG37304                   0040b640     AccessBridgeCalls.obj
 0003:00000658       $SG37306                   0040b658     AccessBridgeCalls.obj
 0003:00000674       $SG37308                   0040b674     AccessBridgeCalls.obj
 0003:00000688       $SG37310                   0040b688     AccessBridgeCalls.obj
 0003:000006a0       $SG37312                   0040b6a0     AccessBridgeCalls.obj
 0003:000006b4       $SG37314                   0040b6b4     AccessBridgeCalls.obj
 0003:000006cc       $SG37316                   0040b6cc     AccessBridgeCalls.obj
 0003:000006e4       $SG37318                   0040b6e4     AccessBridgeCalls.obj
 0003:00000704       $SG37320                   0040b704     AccessBridgeCalls.obj
 0003:00000720       $SG37322                   0040b720     AccessBridgeCalls.obj
 0003:00000738       $SG37324                   0040b738     AccessBridgeCalls.obj
 0003:00000754       $SG37326                   0040b754     AccessBridgeCalls.obj
 0003:0000076c       $SG37328                   0040b76c     AccessBridgeCalls.obj
 0003:00000794       $SG37330                   0040b794     AccessBridgeCalls.obj
 0003:000007bc       $SG37332                   0040b7bc     AccessBridgeCalls.obj
 0003:000007e4       $SG37334                   0040b7e4     AccessBridgeCalls.obj
 0003:00000808       $SG37336                   0040b808     AccessBridgeCalls.obj
 0003:0000082c       $SG37338                   0040b82c     AccessBridgeCalls.obj
 0003:00000850       $SG37340                   0040b850     AccessBridgeCalls.obj
 0003:00000878       $SG37342                   0040b878     AccessBridgeCalls.obj
 0003:000008a0       $SG37344                   0040b8a0     AccessBridgeCalls.obj
 0003:000008c8       $SG37346                   0040b8c8     AccessBridgeCalls.obj
 0003:000008f0       $SG37348                   0040b8f0     AccessBridgeCalls.obj
 0003:00000900       $SG37350                   0040b900     AccessBridgeCalls.obj
 0003:00000914       $SG37352                   0040b914     AccessBridgeCalls.obj
 0003:00000928       $SG37354                   0040b928     AccessBridgeCalls.obj
 0003:00000944       $SG37356                   0040b944     AccessBridgeCalls.obj
 0003:00000954       $SG37358                   0040b954     AccessBridgeCalls.obj
 0003:00000968       $SG37360                   0040b968     AccessBridgeCalls.obj
 0003:00000984       $SG37362                   0040b984     AccessBridgeCalls.obj
 0003:00000994       $SG37364                   0040b994     AccessBridgeCalls.obj
 0003:000009a4       $SG37366                   0040b9a4     AccessBridgeCalls.obj
 0003:000009c0       $SG37368                   0040b9c0     AccessBridgeCalls.obj
 0003:000009d8       $SG37370                   0040b9d8     AccessBridgeCalls.obj
 0003:000009ec       $SG37372                   0040b9ec     AccessBridgeCalls.obj
 0003:00000a00       $SG37374                   0040ba00     AccessBridgeCalls.obj
 0003:00000a14       $SG37376                   0040ba14     AccessBridgeCalls.obj
 0003:00000a28       ?warning@?1??appendToBuffer@@YAHPADI0ZZ@4PADA 0040ba28     AccessInfo.obj
 0003:00000a8c       ?szAppName@?1???0Jaccesswalker@@QAE@H@Z@4PADA 0040ba8c     jaccesswalker.obj
 0003:00000a9c       ?szMenuName@?1???0Jaccesswalker@@QAE@H@Z@4PADA 0040ba9c     jaccesswalker.obj
 0003:00000b70       _logFP                     0040bb70     AccessBridgeDebug.obj
 0003:00000b78       ?retbuf@?1??printError@@9@4PADA 0040bb78     AccessBridgeDebug.obj
 0003:00000c88       ?datebuf@?1??getTimeAndDate@@YAPADXZ@4PADA 0040bc88     AccessInfo.obj
 0003:00000cf8       _GS_ExceptionRecord        0040bcf8     MSVCRT:gs_report.obj
 0003:00000d48       _GS_ContextRecord          0040bd48     MSVCRT:gs_report.obj
 0003:0000101c       ?is_initialized_as_dll@@3_NA 0040c01c     MSVCRT:utility.obj
 0003:0000101d       ?module_local_atexit_table_initialized@@3_NA 0040c01d     MSVCRT:utility.obj
 0003:00001020       ?module_local_atexit_table@@3U_onexit_table_t@@A 0040c020     MSVCRT:utility.obj
 0003:0000102c       ?module_local_at_quick_exit_table@@3U_onexit_table_t@@A 0040c02c     MSVCRT:utility.obj
 0004:000001d0       $R000000                   0040d1d0     jaccesswalker.exe.res
 0004:00000510       $R000340                   0040d510     jaccesswalker.exe.res
 0004:000005a0       $R0003D0                   0040d5a0     jaccesswalker.exe.res
 0004:00000630       $R000460                   0040d630     jaccesswalker.exe.res
 0004:000006d0       $R000500                   0040d6d0     jaccesswalker.exe.res
